:020000040800F2
:100000000080002019980008A14C0008A94C0008A5
:10001000B14C0008B94C0008C14C000800000000B9
:10002000000000000000000000000000C94C0008B3
:10003000D74C000800000000E54C0008F34C000815
:10004000699800086998000869980008699800088C
:10005000699800086998000869980008699800087C
:10006000699800086998000869980008699800086C
:10007000699800086998000869980008699800085C
:10008000699800086998000869980008699800084C
:10009000014D0008154D000869980008699800088E
:1000A000699800086998000869980008699800082C
:1000B000699800086998000869980008699800081C
:1000C000699800086998000869980008699800080C
:1000D00069980008699800086998000869980008FC
:1000E00069980008699800086998000800000000F5
:1000F0000000000000000000000000000000000000
:1001000000000000000000000000000069980008E6
:1001100069980008699800086998000800000000C4
:1001200069980008699800086998000869980008AB
:1001300069980008000000000000000000000000B6
:10014000699800086998000800000000000000009D
:10015000000000000000000000000000000000009F
:10016000000000000000000069980008699800087D
:100170006998000800000000000000000000000076
:0801800000000000699800086E
:1001880081F0004102E000BF83F0004330B54FEA40
:1001980041044FEA430594EA050F08BF90EA020FAD
:1001A8001FBF54EA000C55EA020C7FEA645C7FEA40
:1001B800655C00F0E2804FEA5454D4EB5555B8BF63
:1001C8006D420CDD2C4480EA020281EA030382EAD4
:1001D800000083EA010180EA020281EA0303362D66
:1001E80088BF30BD11F0004F4FEA01314FF4801C39
:1001F8004CEA113102D0404261EB410113F0004F4B
:100208004FEA03334CEA133302D0524263EB430301
:1002180094EA050F00F0A780A4F10104D5F1200E9F
:100228000DDB02FA0EFC22FA05F2801841F10001FA
:1002380003FA0EF2801843FA05F359410EE0A5F1CE
:1002480020050EF1200E012A03FA0EFC28BF4CF0FF
:10025800020C43FA05F3C01851EBE37101F00045B5
:1002680007D54FF0000EDCF1000C7EEB00006EEBC2
:100278000101B1F5801F1BD3B1F5001F0CD349084C
:100288005FEA30004FEA3C0C04F101044FEA4452A3
:1002980012F5800F80F09A80BCF1004F08BF5FEA2A
:1002A800500C50F1000041EB045141EA050130BD0A
:1002B8005FEA4C0C404141EB0101013C28BFB1F51C
:1002C800801FE9D291F0000F04BF01460020B1FA67
:1002D80081F308BF2033A3F10B03B3F120020CDA3A
:1002E8000C3208DD02F1140CC2F10C0201FA0CF018
:1002F80021FA02F10CE002F11402D8BFC2F1200C7D
:1003080001FA02F120FA0CFCDCBF41EA0C01904032
:10031800E41AA2BF01EB0451294330BD6FEA04047B
:100328001F3C1CDA0C340EDC04F11404C4F1200266
:1003380020FA04F001FA02F340EA030021FA04F378
:1003480045EA030130BDC4F10C04C4F1200220FACF
:1003580002F001FA04F340EA0300294630BD21FA0D
:1003680004F0294630BD94F0000F83F4801306BFD3
:1003780081F480110134013D4EE77FEA645C18BFC7
:100388007FEA655C29D094EA050F08BF90EA020F5E
:1003980005D054EA000C04BF1946104630BD91EA56
:1003A800030F1EBF0021002030BD5FEA545C05D159
:1003B8004000494128BF41F0004130BD14F5800498
:1003C8003CBF01F5801130BD01F0004545F0FE410C
:1003D80041F470014FF0000030BD7FEA645C1ABF41
:1003E800194610467FEA655C1CBF0B46024650EA78
:1003F800013406BF52EA033591EA030F41F40021A4
:1004080030BD00BF90F0000F04BF0021704730B529
:100418004FF4806404F132044FF000054FF00001FE
:1004280050E700BF90F0000F04BF0021704730B5BF
:100438004FF4806404F1320410F0004548BF404294
:100448004FF000013EE700BF42004FEAE2014FEAE9
:1004580031014FEA02701FBF12F07F4393F07F4FC4
:1004680081F06051704732F07F4208BF704793F0C7
:100478007F4F04BF41F40021704730B54FF46074DA
:1004880001F0004521F000411CE700BF50EA0102DD
:1004980008BF704730B54FF000050AE050EA010286
:1004A80008BF704730B511F0004502D5404261EBF6
:1004B80041014FF4806404F132045FEA915C3FF437
:1004C800D8AE4FF003025FEADC0C18BF03325FEAD4
:1004D800DC0C18BF033202EBDC02C2F1200300FA85
:1004E80003FC20FA02F001FA03FE40EA0E0021FAAA
:1004F80002F11444BDE600BF70B54FF0FF0C4CF498
:10050800E06C1CEA11541DBF1CEA135594EA0C0F49
:1005180095EA0C0F00F0DEF82C4481EA030621EA84
:100528004C5123EA4C5350EA013518BF52EA0335BF
:1005380041F4801143F4801338D0A0FB02CE4FF071
:100548000005E1FB02E506F00042E0FB03E54FF0A1
:100558000006E1FB03569CF0000F18BF4EF0010E99
:10056800A4F1FF04B6F5007F64F5407404D25FEA95
:100578004E0E6D4146EB060642EAC62141EA555148
:100588004FEAC52040EA5E504FEACE2EB4F1FD0C8A
:1005980088BFBCF5E06F1ED8BEF1004F08BF5FEA08
:1005A800500E50F1000041EB045170BD06F00046BA
:1005B80046EA010140EA020081EA0301B4EB5C0467
:1005C800C2BFD4EB0C0541EA045170BD41F480115F
:1005D8004FF0000E013C00F3AB8014F1360FDEBF84
:1005E800002001F0004170BDC4F10004203C35DA60
:1005F8000C341BDC04F11404C4F1200500FA05F3E3
:1006080020FA04F001FA05F240EA020001F0004283
:1006180021F0004110EBD37021FA04F642EB0601F9
:100628005EEA430E08BF20EAD37070BDC4F10C0423
:10063800C4F1200500FA04F320FA05F001FA04F2E7
:1006480040EA020001F0004110EBD37041F10001D3
:100658005EEA430E08BF20EAD37070BDC4F12005DE
:1006680000FA05F24EEA020E20FA04F301FA05F246
:1006780043EA020321FA04F001F0004121FA04F2EE
:1006880020EA020000EBD3705EEA430E08BF20EABE
:10069800D37070BD94F0000F0FD101F000464000F8
:1006A80041EB010111F4801F08BF013CF7D041EA7A
:1006B800060195F0000F18BF704703F0004652007E
:1006C80043EB030313F4801F08BF013DF7D043EA4F
:1006D8000603704794EA0C0F0CEA135518BF95EA05
:1006E8000C0F0CD050EA410618BF52EA4306D1D18C
:1006F80081EA030101F000414FF0000070BD50EAAB
:10070800410606BF1046194652EA430619D094EA34
:100718000C0F02D150EA013613D195EA0C0F05D11E
:1007280052EA03361CBF104619460AD181EA030172
:1007380001F0004141F0FE4141F470014FF000002A
:1007480070BD41F0FE4141F4780170BD70B54FF0C5
:10075800FF0C4CF4E06C1CEA11541DBF1CEA135545
:1007680094EA0C0F95EA0C0F00F0A7F8A4EB050427
:1007780081EA030E52EA03354FEA013100F088801E
:100788004FEA03334FF0805545EA131343EA1263E7
:100798004FEA022245EA111545EA10654FEA00269C
:1007A8000EF000419D4208BF964244F1FD0404F555
:1007B800407402D25B084FEA3202B61A65EB0305B1
:1007C8005B084FEA32024FF480104FF4002CB6EB6E
:1007D800020E75EB030E22BFB61A754640EA0C00EE
:1007E8005B084FEA3202B6EB020E75EB030E22BF2E
:1007F800B61A754640EA5C005B084FEA3202B6EB6F
:10080800020E75EB030E22BFB61A754640EA9C002D
:100818005B084FEA3202B6EB020E75EB030E22BFFD
:10082800B61A754640EADC0055EA060E18D04FEABB
:10083800051545EA16754FEA06164FEAC30343EA5B
:1008480052734FEAC2025FEA1C1CC0D111F4801F28
:100858000BD141EA00014FF000004FF0004CB6E721
:1008680011F4801F04BF01430020B4F1FD0C88BFC0
:10087800BCF5E06F3FF6AFAEB5EB030C04BFB6EBCB
:10088800020C5FEA500C50F1000041EB045170BDBE
:100898000EF0004E4EEA113114EB5C04C2BFD4EBEB
:1008A8000C0541EA045170BD41F480114FF0000E6F
:1008B800013C90E645EA060E8DE60CEA135594EAEB
:1008C8000C0F08BF95EA0C0F3FF43BAF94EA0C0FEE
:1008D8000AD150EA01347FF434AF95EA0C0F7FF463
:1008E80025AF104619462CE795EA0C0F06D152EAB7
:1008F80003353FF4FDAE1046194622E750EA41069B
:1009080018BF52EA43067FF4C5AE50EA41047FF4AB
:100918000DAF52EA43057FF4EBAE12E74FEA41020E
:1009280012F5001215D211D56FF47873B3EB625239
:1009380012D94FEAC12343F0004343EA505311F060
:10094800004F23FA02F018BF404270474FF00000F2
:10095800704750EA013005D111F0004008BF6FF030
:10096800004070474FF00000704700BF4A0011D2A6
:1009780012F5001211D20DD56FF47873B3EB6252F1
:100988000ED44FEAC12343F0004343EA505323FAFD
:1009980002F070474FF00000704750EA013002D172
:1009A8004FF0FF3070474FF0000070474FEA4102A8
:1009B800B2F1E04324BFB3F5001CDCF1FE5C0DD9B5
:1009C80001F0004C4FEAC0024CEA5070B2F1004FFF
:1009D80040EB830008BF20F00100704711F0804F02
:1009E80021D113F13872BCBF01F00040704741F4C7
:1009F80080114FEA5252C2F11802C2F1200C10FACB
:100A08000CF320FA02F018BF40F001004FEAC123AE
:100A18004FEAD32303FA0CFC40EA0C0023FA02F352
:100A28004FEA4303CCE77FEA625307D150EA013328
:100A38001EBF4FF0FE4040F44000704701F00040F8
:100A480040F0FE4040F40000704700BF0348044BEC
:100A5800834202D0034B03B1184770476800002057
:100A680068000020000000000548064B1B1AD90F3B
:100A780001EBA301491002D0034B03B1184770479B
:100A880068000020680000200000000010B5064C37
:100A9800237843B9FFF7DAFF044B13B10448AFF3E7
:100AA80000800123237010BD6800002000000000B2
:100AB8001099000808B5054B1BB105490548AFF367
:100AC8000080BDE80840FFF7CFBF00BF000000006E
:100AD8006C0000201099000880B584B000AF7860E1
:100AE8000C4A7B6813600B4B1B680221184604F004
:100AF800AEFD0346FB73FB7B002B01D0FB7B05E0BF
:100B0800044B1B68184604F06CFB03461846103764
:100B1800BD4680BD8400002080B586B000AF034686
:100B2800B9607A60FB81FB890B4A13600A4B00228B
:100B38009A60094B0022DA60074A7B681361074B09
:100B4800186807F11403BA68034904F08EFB0346DA
:100B580018461837BD4680BD880000208400002054
:100B680080B584B000AF03460A46FB801346BB80BD
:100B7800264B1B6803F00103002B10D1FB885B0197
:100B8800234A1360BB885B01214A9360FB885B01A1
:100B98001F4A5360BB885B011D4AD36007E0FB888E
:100BA8005B011B4A5360BB885B01194AD360184B31
:100BB80000221A61154B1B685B08154A5361144BD8
:100BC8005B690E2B01D901231CE0114B00229A61AD
:100BD8000F4B0022DA610E4B01221A620C4B0D22D8
:100BE8005A620C4B1B680A49184604F030FA03464F
:100BF800FB73FB7B002B04D1044B1B680133034AB6
:100C08001360FB7B18461037BD4680BDA00000204E
:100C1800A40000208400002080B58CB000AF78606C
:100C2800124B1B687A689A4217D1104B186807F163
:100C38000C0307F11402002104F0E7FB0346002B24
:100C48000DD1FB69002B0CD17B699BB2796A07F146
:100C58000C02184602F07AF904E000BF02E000BF77
:100C680000E000BF3037BD4680BD00BF84000020D3
:100C780080B487B000AFF860C7E900233B6A082B4F
:100C880001D908233B623B6A013B7B6113E07B6926
:100C9800FA6813443A781A70D7E900014FF0000255
:100CA8004FF00003020A42EA01620B0AC7E9002377
:100CB8007B69013B7B617B69002BE8DAFA683B6A58
:100CC800134418461C37BD465DF8047B7047000086
:100CD80080B584B000AF00F073F80022002127200F
:100CE80001F02BFA0A2001F08BFB00F069F800F004
:100CF800CBFB40F2A11140F2654000F0CFFB214A46
:100D08003B1D92E803001860043319803B1D06223E
:100D1800194640F2177001F083F90346FB73FB7B19
:100D2800002B01D0FB7B28E03B1D0622194640F230
:100D3800157001F075F90346BB73BB7B002B01D01E
:100D4800BB7B1AE0002200214FF4787001F068F9AB
:100D580003467B737B7B002B01D07B7B0DE000225D
:100D680000214FF4826001F05BF903463B733B7B43
:100D7800002B01D03B7B00E0002318461037BD460E
:100D880080BD00BF2899000880B582B000AF7860A8
:100D98000B46FB701346BB70786800F0C5FE064A28
:100DA800FB781370054ABB781370FFF791FF034671
:100DB80018460837BD4680BDCC000020CD00002075
:100DC80080B582B000AF3B4606221946022001F0EA
:100DD800B4F9034618460837BD4680BD80B582B0D1
:100DE80000AF7860786800F003FC034618460837BF
:100DF800BD4680BD0000000080B588B000AF7860B7
:100E080007F1100300221A609A8007F110030622E6
:100E18001946322001F091F90346FB77FB7F002B3E
:100E280001D0FB7F22E33B7C1AB27B7C1BB21B0206
:100E38001BB213431BB29AB27B68A3F84820BB7C51
:100E48001AB2FB7C1BB21B021BB213431BB2C3F3C7
:100E58000C0399B27A68B2F84A3061F3CF03A2F86A
:100E68004A303B7DDB09DBB203F00103D9B27A6873
:100E780092F84C3061F3000382F84C303B7D9B09BB
:100E8800DBB203F00103D9B27A6892F84C3061F30F
:100E9800410382F84C303B7D5B09DBB203F0010370
:100EA800D9B27A6892F84C3061F3820382F84C30F8
:100EB8003B7D1B09DBB203F00103D9B27A6892F8D3
:100EC8004C3061F3C30382F84C303B7DDB08DBB266
:100ED80003F00103D9B27A6892F84C3061F3041335
:100EE80082F84C303B7D9B08DBB203F00103D9B29A
:100EF8007A6892F84C3061F3451382F84C303B7DA8
:100F08005B08DBB203F00103D9B27A6892F84C307F
:100F180061F3861382F84C303B7D03F00103D9B2AC
:100F28007A6892F84C3061F3C71382F84C307B7DB5
:100F3800DB09DBB203F00103D9B27A6892F84D30CD
:100F480061F3000382F84D307B7D9B09DBB203F02F
:100F58000103D9B27A6892F84D3061F3410382F8FF
:100F68004D307B7D5B09DBB203F00103D9B27A68AF
:100F780092F84D3061F3820382F84D307B7D1B0976
:100F8800DBB203F00103D9B27A6892F84D3061F30D
:100F9800C30382F84D307B7DDB08DBB203F001032D
:100FA800D9B27A6892F84D3061F3041382F84D3063
:100FB8007B7D9B08DBB203F00103D9B27A6892F813
:100FC8004D3061F3451382F84D307B7D5B08DBB211
:100FD80003F00103D9B27A6892F84D3061F38613B1
:100FE80082F84D307B7D03F00103D9B27A6892F81C
:100FF8004D3061F3C71382F84D3040F21E7001F096
:1010080049F90346002B01D100232FE207F1100311
:1010180006221946192001F090F80346BB77BB7FDA
:10102800002B01D0BB7F21E23B7C1AB27B7C1BB238
:101038001B021BB213431BB21846FFF7F3F90FF25A
:101048003843D3E90023FFF757FA02460B46104608
:1010580019460FF22C43D3E90023FFF797F802460D
:101068000B4610461946FFF7A1FC02467B681A6238
:10107800BB7C1AB2FB7C1BB21B021BB213431BB214
:101088001846FFF7CFF9FCA3D3E90023FFF734FA9A
:1010980002460B4610461946F9A3D3E90023FFF789
:1010A80075F802460B4610461946FFF77FFC0246C4
:1010B8007B685A623B7D1AB27B7D1BB21B021BB256
:1010C80013431BB21846FFF7ADF9EBA3D3E900238E
:1010D800FFF712FA02460B4610461946E8A3D3E971
:1010E8000023FFF753F802460B4610461946FFF750
:1010F8005DFC02467B689A6207F1100306221946D6
:101108001A2001F01AF803467B777B7F002B01D069
:101118007B7FABE13B7C1AB27B7C1BB21B021BB210
:1011280013431BB21846FFF77DF9D3A3D3E9002375
:10113800FFF7E2F902460B4610461946D0A3D3E959
:101148000023FFF723F802460B4610461946FFF71F
:101158002DFC02467B68DA62BB7C1AB2FB7C1BB2B0
:101168001B021BB213431BB21846FFF75BF9C2A35D
:10117800D3E90023FFF7C0F902460B46104619468B
:10118800BFA3D3E90023FFF701F802460B46104638
:101198001946FFF70BFC02467B681A633B7D1AB2BF
:1011A8007B7D1BB21B021BB213431BB21846FFF711
:1011B80039F9B1A3D3E90023FFF79EF902460B469C
:1011C80010461946AEA3D3E90023FEF7DFFF024617
:1011D8000B4610461946FFF7E9FB02467B685A633F
:1011E80007F11003062219461B2000F0A6FF03464C
:1011F8003B773B7F002B01D03B7F37E13B7C1AB22A
:101208007B7C1BB21B021BB213431BB21846FFF7B1
:1012180009F999A3D3E90023FFF76EF902460B46B3
:101228001046194696A3D3E90023FEF7AFFF0246FE
:101238000B4610461946FFF7B9FB02467B689A63CE
:10124800BB7C1AB2FB7C1BB21B021BB213431BB242
:101258001846FFF7E7F888A3D3E90023FFF74CF90E
:1012680002460B461046194685A3D3E90023FEF72C
:101278008DFF02460B4610461946FFF797FB0246BC
:101288007B68DA633B7D1AB27B7D1BB21B021BB203
:1012980013431BB21846FFF7C5F877A3D3E9002319
:1012A800FFF72AF902460B461046194674A3D3E9FC
:1012B8000023FEF76BFF02460B4610461946FFF760
:1012C80075FB02467B681A6407F11003062219466B
:1012D8001F2000F032FF0346FB76FB7E002B01D077
:1012E800FB7EC3E03B7C1AB27B7C1BB21B021BB2A9
:1012F80013431BB21846FFF795F85FA3D3E9002301
:10130800FFF7FAF802460B46104619465CA3D3E9E4
:101318000023FEF73BFF02460B4610461946FFF72F
:1013280045FB02467B685A6407F108030622194602
:10133800302000F002FF0346BB76BB7E002B01D0B5
:10134800BB7E93E0BB7A1AB2FB7A1BB21B021BB2BC
:1013580013431BB29AB27B68A3F84E2007F1080327
:1013680006221946312000F0E8FE03467B767B7E94
:10137800002B01D07B7E79E03B7A1AB27B7A1BB2D4
:101388001B021BB213431BB21846FFF74BF83AA3D4
:10139800D3E90023FFF7B0F802460B46104619467A
:1013A80037A3D3E90023FEF7F1FE02460B461046A9
:1013B8001946FFF7DBFA03469AB27B68A3F8522076
:1013C800BB7A1AB2FB7A1BB21B021BB213431BB2C5
:1013D8001846FFF727F828A3D3E90023FFF78CF86E
:1013E80002460B461046194625A3D3E90023FEF70B
:1013F800CDFE02460B4610461946FFF7B7FA0346DC
:101408009AB27B68A3F850203B7B1AB27B7B1BB255
:101418001B021BB213431BB21846FFF703F816A3AF
:10142800D3E90023FFF768F802460B461046194631
:1014380013A3D3E90023FEF7A9FE02460B46104684
:101448001946FFF793FA03469AB27B68A3F8562029
:10145800002200214FF4826000F0E2FD03463B7653
:101468003B7E002B01D03B7E00E00023184620374E
:10147800BD4680BDAFF30080333333333333C33FCE
:10148800000000000070974080B500AF00220021E6
:10149800282000F0C5FD0346184680BD80B584B0FD
:1014A80000AF03460A46FB801346BB80BB8803F4A3
:1014B8007043002B04D1FB8803F47043002B01D048
:1014C80001233CE007F1080306221946262000F014
:1014D80034FE0346FB73FB7B002B01D0FB7B2EE025
:1014E800BB88DBB23B727B7A23F00F03DBB27B72E3
:1014F8007B7A5AB2BB881B0A9BB25BB203F00F031C
:101508005BB213435BB2DBB27B727B7A03F00F03EF
:10151800DBB27B727A7AFB88DBB21B01DBB2134346
:10152800DBB27B72FB881B099BB2DBB2BB7207F193
:10153800080306221946242000F072FD03461846C7
:101548001037BD4680BD000080B586B000AF78601A
:1015580000233B6107F1080306221946332000F0F7
:10156800ECFD0346FB73FB7B002B01D0FB7B37E0D4
:101578003B7A1A467B7A1B021A43BB7A1B041A432E
:10158800FB7A1B0613433B617B680022DA667B68A3
:1015980000221A6700237B611BE07B681A6F7B6956
:1015A8005B00396921FA03F303F001031A437B68EE
:1015B8001A677B68DA6E7B695B000133396921FA47
:1015C80003F303F001031A437B68DA667B6901338E
:1015D8007B61054B1B781A467B699342DDD3002358
:1015E80018461837BD4680BDCC000020000000001A
:1015F80080B586B000AF786007F10C030622194663
:10160800042000F09AFD0346FB75FB7D002B01D0FA
:10161800FB7D7CE23B7B1AB27B7B1BB21B021BB2BD
:1016280013431BB21846FEF7FDFE0FF2EC43D3E955
:101638000023FEF761FF02460B46104619460FF2DB
:10164800E043D3E90023FEF7A1FD02460B4610460E
:101658001946FFF763F903461AB27B681A80BB7B09
:101668001AB2FB7B1BB21B021BB213431BB21846F8
:10167800FEF7D8FE0FF2A043D3E90023FEF73CFFA4
:1016880002460B46104619460FF29443D3E900234D
:10169800FEF77CFD02460B4610461946FFF73EF959
:1016A80003461AB27B685A803B7C1AB27B7C1BB219
:1016B8001B021BB213431BB21846FEF7B3FE0FF210
:1016C8005843D3E90023FEF717FF02460B4610469E
:1016D80019460FF24C43D3E90023FEF757FD0246A3
:1016E8000B4610461946FFF719F903461AB27B68EC
:1016F8009A8007F10C0306221946062000F01DFD0A
:101708000346BB75BB7D002B01D0BB7DFFE13B7B56
:101718001AB27B7B1BB21B021BB213431BB21846C7
:10172800FEF780FEFCA3D3E90023FEF7E5FE0246A0
:101738000B4610461946FAA3D3E90023FEF726FD07
:1017480002460B4610461946FFF7E8F803461AB258
:101758007B68DA80BB7B1AB2FB7B1BB21B021BB215
:1017680013431BB21846FEF75DFEEBA3D3E9002333
:10177800FEF7C2FE02460B4610461946E8A3D3E917
:101788000023FEF703FD02460B4610461946FFF7F5
:10179800C5F803461AB27B681A813B7C1AB27B7C77
:1017A8001BB21B021BB213431BB21846FEF73AFECC
:1017B800D9A3D3E90023FEF79FFE02460B46104645
:1017C8001946D7A3D3E90023FEF7E0FC02460B46EF
:1017D80010461946FFF7A2F803461AB27B685A81E9
:1017E80007F10C0306221946082000F0A6FC034660
:1017F8007B757B7D002B01D07B7D88E13B7B1AB21A
:101808007B7B1BB21B021BB213431BB21846FEF7AD
:1018180009FEC1A3D3E90023FEF76EFE02460B467C
:1018280010461946BEA3D3E90023FEF7AFFC0246D3
:101838000B4610461946FFF771F803461AB27B6843
:101848009A81BB7B1AB2FB7B1BB21B021BB21343F0
:101858001BB21846FEF7E6FDAFA3D3E90023FEF757
:101868004BFE02460B4610461946ADA3D3E90023AA
:10187800FEF78CFC02460B4610461946FFF74EF859
:1018880003461AB27B68DA813B7C1AB27B7C1BB2B6
:101898001B021BB213431BB21846FEF7C3FD9EA3DF
:1018A800D3E90023FEF728FE02460B4610461946E8
:1018B8009BA3D3E90023FEF769FC02460B461046BA
:1018C8001946FFF72BF803461AB27B681A8207F10C
:1018D8000C03062219460A2000F02FFC03463B752C
:1018E8003B7D002B01D03B7D11E13B7B1AB27B7B1A
:1018F8001BB21B021BB213431BB21846FEF792FD24
:1019080085A3D3E90023FEF7F7FD02460B461046F0
:10191800194683A3D3E90023FEF738FC02460B4699
:1019280010461946FEF7FAFF03461AB27B685A8238
:10193800BB7B1AB2FB7B1BB21B021BB213431BB24D
:101948001846FEF76FFD74A3D3E90023FEF7D4FD14
:1019580002460B461046194671A3D3E90023FEF749
:1019680015FC02460B4610461946FEF7D7FF0346FC
:101978001AB27B689A823B7C1AB27B7C1BB21B0230
:101988001BB213431BB21846FEF74CFD62A3D3E902
:101998000023FEF7B1FD02460B461046194660A328
:1019A800D3E90023FEF7F2FB02460B461046194620
:1019B800FEF7B4FF03461AB27B68DA8207F10C031C
:1019C80006221946092000F0B8FB0346FB74FB7C8D
:1019D800002B01D0FB7C9AE03B7B1AB27B7B1BB2CD
:1019E8001B021BB213431BB21846FEF71BFD4AA38A
:1019F800D3E90023FEF780FD02460B461046194640
:101A080047A3D3E90023FEF7C1FB02460B46104665
:101A18001946FEF783FF03461AB27B681A83BB7B1D
:101A28001AB2FB7B1BB21B021BB213431BB2184634
:101A3800FEF7F8FC38A3D3E90023FEF75DFD024664
:101A48000B461046194636A3D3E90023FEF79EFB42
:101A580002460B4610461946FEF760FF03461AB2C7
:101A68007B685A833B7C1AB27B7C1BB21B021BB27D
:101A780013431BB21846FEF7D5FC27A3D3E900236E
:101A8800FEF73AFD02460B461046194624A3D3E951
:101A98000023FEF77BFB02460B4610461946FEF76D
:101AA8003DFF03461AB27B689A8307F10C030622AE
:101AB80019460B2000F041FB0346BB74BB7C002B8E
:101AC80001D0BB7C23E03B7B1AB27B7B1BB21B02A1
:101AD8001BB213431BB21846FEF7A4FC0EA3D3E9AE
:101AE8000023FEF709FD02460B46104619460CA3D3
:101AF800D3E90023FEF74AFB02460B461046194677
:101B0800FEF70CFF03461AB27B68DA8300231846F7
:101B18001837BD4680BD00BF333333333333C33F3B
:101B2800000000000070974080B582B000AF786078
:101B380000F0E5FB012003F06BF900F0EAFB044A32
:101B48007B681360002318460837BD4680BD00BF78
:101B5800D000002080B586B000AF78600B46FB70DF
:101B68001023FB82FB78022B38D900233B611CE051
:101B78000023FB6013E03B697A6813441B781A461C
:101B8800FB6802FA03F3FB72FA7AFB8A11461846DD
:101B980000F029F80346FB82FB680133FB60FB6811
:101BA800072BE8DD3B6901333B61FB78023B3A696F
:101BB8009A42DDDBFB8ADB0999B2FB78023B7A6843
:101BC8001344CAB21A70FB8ADAB2FB78013B79680F
:101BD8000B445200D2B21A70002300E001231846C9
:101BE8001837BD4680BD80B487B000AF03460A46AB
:101BF800FB8013467B717B79DB097B71FB889B0B30
:101C08009BB25BB203F001035AB297F90530534017
:101C18005BB2FB75FB889B089BB25BB203F00103C8
:101C28005AB297F9173053405BB2BB75FB88DB0893
:101C38009BB25BB203F001035AB297F917305340D5
:101C48005BB27B75FB889B099BB25BB203F0010317
:101C58005AB297F9173053405BB23B75FB88DB09E2
:101C68009BB25BB203F001035AB297F917305340A5
:101C78005BB2FB74FB885B0A9BB25BB203F00103A7
:101C88005AB297F9173053405BB2BB74FB885B0BB1
:101C98009BB25BB203F001035AB297F91730534075
:101CA8005BB27B740023FB817B7C1BB29B031AB263
:101CB800B7F90E3013431BB2FB81B7F906305B004E
:101CC8001BB203F400531AB2B7F90E3013431BB218
:101CD800FB81B7F906305B001BB203F480531AB2DC
:101CE800B7F90E3013431BB2FB81B7F906305B001E
:101CF8001BB203F400631AB2B7F90E3013431BB2D8
:101D0800FB81BB7C1BB29B021AB2B7F90E3013439E
:101D18001BB2FB81B7F906305B001BB203F40073FA
:101D28001AB2B7F90E3013431BB2FB81FB7C1BB20E
:101D38001B021AB2B7F90E3013431BB2FB813B7D6D
:101D48001BB2DB011AB2B7F90E3013431BB2FB8189
:101D5800B7F906305B001BB203F040031AB2B7F9BB
:101D68000E3013431BB2FB81B7F906305B001BB280
:101D780003F020031AB2B7F90E3013431BB2FB81EC
:101D88007B7D1BB21B011AB2B7F90E3013431BB28D
:101D9800FB81BB7D1BB2DB001AB2B7F90E301343CF
:101DA8001BB2FB81B7F906305B001BB203F00403DA
:101DB8001AB2B7F90E3013431BB2FB81B7F90630DC
:101DC8005B001BB203F002031AB2B7F90E301343DB
:101DD8001BB2FB81FB7D9AB2FB891343FB81FB8914
:101DE80018461C37BD465DF8047B704780B487B041
:101DF80000AF0346B9607A60FB731023FB828F2320
:101E08003B8200237B7524E07B7D7A6813441B7832
:101E18009B009AB2FB8A5340FB8208233B7512E071
:101E2800FB8A03F40073002B07DDFB8A5B00FB824F
:101E3800FA8A3B8A5340FB8202E0FB8A5B00FB8202
:101E48003B7D013B3B753B7D002BE9D17B7D01331D
:101E58007B757B7DBA689A42D6DCFB7B002B27D04A
:101E6800BB687A6813441B781BB29B001BB203F44F
:101E78007C731AB2B7F9163053401BB2FB820623A3
:101E8800FB7412E0FB8A03F40073002B07DDFB8A66
:101E98005B00FB82FA8A3B8A5340FB8202E0FB8AA2
:101EA8005B00FB82FB7C013BFB74FB7C002BE9D1D4
:101EB800FB8AC3F309039BB218461C37BD465DF87D
:101EC800047B704780B584B000AF78600B46FB7028
:101ED800FB78022B1CD9FB78023B7A681946012053
:101EE800FFF784FF0346C3F30903FB81FB891B0A41
:101EF80099B2FB78023B7A681344CAB21A70FB782D
:101F0800013B7A681344FA89D2B21A70002300E0C0
:101F1800012318461037BD4680BD80B584B000AF98
:101F280078600B46FB70FB78022B01D8FF230DE08D
:101F3800FB789BB21946786800F03AF80346FB81B3
:101F4800FB89002B14BF01230023DBB2184610378E
:101F5800BD4680BD80B485B000AF0346FB71002349
:101F6800FB8100237B73FB799BB29B00FB810023E1
:101F78007B7313E0FB8903F40073002B08D0B7F9D7
:101F88000E305B001BB283F08F031BB2FB8102E0B3
:101F9800FB895B00FB817B7B01337B737B7B072B9E
:101FA800E8D9FB8918461437BD465DF8047B7047AD
:101FB80090B585B000AF78600B467B801023FB811D
:101FC8000023BB810023BB811CE0B7F90E301B0244
:101FD8001CB2FB899B089BB2DAB2B7F90C3079685E
:101FE8000B441B785340DBB21846FFF7B3FF034698
:101FF8001BB263401BB2FB81B7F90C309BB20133B3
:102008009BB2BB81B7F90C207B889A42DDDBFB8948
:10201800C3F30903FB81FB8918461437BD4690BDFD
:102028002DE9F04387B000AF03463960FB801346C3
:102038007B717B79002B60D06B461E467B79991D9E
:102048004B1E3B610A460023904699464FF000021A
:102058004FF000034FEAC90343EA58734FEAC80236
:102068000A46002314461D464FF000024FF00003B5
:10207800EB0043EA5473E2000B460733DB08DB004E
:10208800ADEB030D6B460033FB60FB881B0A9BB26C
:10209800DAB2FB681A70FB88DAB2FB685A7004215E
:1020A800F868FFF757FD0023BB750AE0BB7D3A6867
:1020B8001A44BB7D04331178FA68D154BB7D0133CF
:1020C800BB75BA7D7B799A42F0D3FB681A1D7B7980
:1020D8000233DBB219461046FFF7F4FE00F00FF9A1
:1020E8007B790633DBB21946F86800F01DF9034620
:1020F800FB7500F00EF9B54619E0FB881B0A9BB288
:10210800DBB23B72FB88DBB27B7207F10803042168
:102118001846FFF71FFD00F0F2F807F10803042145
:10212800184600F001F90346FB7500F0F2F8FB7D54
:1021380018461C37BD46BDE8F0832DE9F04F8DB039
:1021480000AF03463961FB8213467B756B467B60A3
:102158007B7D991D4B1EBB620A460023BA60FB605B
:102168004FF000024FF00003F868C300B86843EA74
:102178005073B868C2000A46002392469B464FF047
:1021880000024FF000034FEACB0343EA5A734FEAC9
:10219800CA020B460733DB08DB00ADEB030D6B46C9
:1021A80000337B627B7D9E1D731E3B62324600239B
:1021B800904699464FF000024FF000034FEAC903DA
:1021C80043EA58734FEAC8023246002314461D46B4
:1021D8004FF000024FF00003EB0043EA5473E200B3
:1021E80033460733DB08DB00ADEB030D6B460033EA
:1021F800FB61FB8A1B0A9BB2DAB27B6A1A70FB8A04
:10220800DAB27B6A5A700421786AFFF7A3FC00F0FF
:1022180076F87B7D0633DBB21A46796AF86900F0F6
:10222800D5F80346FB7600F074F8FB7E002B01D04E
:10223800FB7E28E0002387F82F300EE097F82F3038
:102248001A1D97F82F3039690B44F9698A5C1A709E
:1022580097F82F30013387F82F3097F82F207B7DA0
:102268009A42EBD33346023BFA69D35C23F003036B
:10227800BB76FB691A1D7B7D0233DBB2194610461B
:10228800FFF74BFE0346D7F804D018463437BD464F
:10229800BDE8F08F80B586B000AF0346FB8007F13C
:1022A800100300221A601A7107F1080300221A604D
:1022B8001A71FB881B0A9BB2DBB23B74FB88DBB24A
:1022C8007B7407F1100304211846FFF743FC00F064
:1022D80016F807F1100107F108030522184600F067
:1022E80075F80346FB7500F014F8FB7D002B01D050
:1022F800FB7D00E03B7B18461837BD4680BD80B5A6
:1023080000AF002210214FF0904003F081FE00BF83
:1023180080BD80B500AF012210214FF0904003F03E
:1023280077FE00BF80BD00002DE9F04389B002AF01
:1023380078600B46FB706B461E46F9780B46013BEE
:102348007B61CBB20022984691464FF000024FF0D5
:1023580000034FEAC90343EA58734FEAC802CBB2F5
:1023680000221C4615464FF000024FF00003EB0018
:1023780043EA5473E2000B460733DB08DB00ADEB9E
:10238800030D02AB00333B610F4B1868FB789BB21F
:10239800642200923A69796806F019F80346FB73DB
:1023A8000023BB60084B1B681B68DB68BB60064BDF
:1023B8001B681B689B68BB60BB68FB7BB5461846FF
:1023C8001C37BD46BDE8F083D000002080B588B03A
:1023D80002AFF860B9601346FB71084B1868FB79C7
:1023E8009BB264220092FA68B96805F0F0FF0346D0
:1023F800FB75FB7D18461837BD4680BDD000002010
:1024080080B582B000AF0346FB80FB88184602F017
:10241800FFFC00BF0837BD4680BD000090B585B001
:1024280000AF7860104B1B78104A1278194678680C
:10243800FEF7AAFC0E4B40F265421A800D4B40F2A3
:10244800A1121A8002F0D8FC044602F0D5FC03461B
:10245800094A1460084A5360084B01221A7000BFE9
:102468001437BD4690BD00BF000000204C0100207D
:102478004A01002048010020540100204F0100209B
:1024880080B500AF224B1A78224B1B789A4219D09C
:102498001F4B1B78062B11D801A252F823F000BF5E
:1024A800C5240008C5240008C5240008C524000860
:1024B800C5240008C5240008C5240008144B1A7850
:1024C800144B1A70124B1B78062B1ED801A252F817
:1024D80023F000BF11250008F9240008FF24000894
:1024E80005250008112500080B25000811250008FE
:1024F80000F012F809E000F00FF806E000F00CF820
:1025080003E000F047F900E000BF00BF80BD00BF56
:102518004F010020500100202DE9B04F88B002AFD4
:10252800FEF74EFC0346002B05D1934B07225A8039
:10253800202000F067FD9148FEF75EFC03461A462E
:102548008F4B1B781344DAB28D4B1A708B4B93F870
:102558004D3003F01003DBB2002B12D0894B1B78EF
:102568000133DAB2874B1A70864B1B78032B06D9D6
:10257800814B07225A80202000F044FD01E0FEF73D
:10258800A7FB7E4BB3F84830002B37D17B4B93F831
:102598004D3003F00803DBB2002B2FD1774B93F8B3
:1025A8004C3003F02003DBB2002B27D1734B93F898
:1025B8004C3023F07F03DBB2002B1FD16F4B93F815
:1025C8004D3003F00203DBB2002B17D16B4B93F8AD
:1025D8004D3003F00103DBB2002B0FD1674B93F8AA
:1025E8004D3023F07F03DBB2002B07D1634B93F808
:1025F8004D3003F04003DBB2002B05D05E4B0A22BE
:102608005A80202000F0FEFC5C4B93F84D3003F01C
:102618002003DBB2002B05D0574B09225A8020201B
:1026280000F0F0FC5548FEF7D9FB03461A46544B18
:102638001B781344DAB2524B1A705048FEF784FFE5
:1026480003461A464E4B1B781344DAB24C4B1A70A9
:102658004B4B1B78052B05D9474B08225A80202065
:1026680000F0D0FC00237B6100233B6148E0434A33
:102678003B6932F91330B3F5486F1BDA01237B61EC
:102688003D4B03225A803B69DAB23B4B1A713E4BF1
:102698007B603A4A3B6932F913301BB2DA17984625
:1026A80091460223009342464B467868FEF7E0FACB
:1026B800786022E0314A3B6932F9133041F268020E
:1026C80093421ADD01237B612B4B02225A803B691E
:1026D800DAB2294B1A712C4BBB60284A3B6932F994
:1026E80013301BB2DA179A469346022300935246D8
:1026F8005B46B868FEF7BCFAB8603B6901333B61DA
:10270800224B1B781A463B699342B0D31B4BB3F854
:102718004E3046F66052934217D9174B09225A8019
:102728001B4BFB60154BB3F84E309BB200221C4686
:1027380015460223009322462B46F868FEF798FABE
:10274800F860202000F05EFC02E0202000F07CFC15
:102758007B69002B03D0012000F054FC02E001202B
:1027680000F072FC0A20FFF74BFE002318461837CA
:10277800BD46BDE8B08F00BFB4010020D4000020E2
:102788004D0100204E010020B9010020000000206A
:10279800B801002080B400AF00231846BD465DF89C
:1027A800047B704780B584B000AFF860B9607A6088
:1027B800144B00221A70144B00221A70134AFB683B
:1027C8001360134ABB681360124A7B6813600F4B8F
:1027D8001B680821184606F0D9F90C4B1B680C2118
:1027E800184606F0D3F9094B1B681B6800225A6388
:1027F800064B1B681B6800229A6300BF1037BD4652
:1028080080BD00BF6C0400206D0400205C01002026
:10281800600100206401002080B485B000AF034649
:10282800FB71FB79642B11D9174B1B681B680022BD
:10283800DA63154B1B681B6800221A64134B0022CD
:102848001A70124B1A78124B1A7018E00F4AFB795B
:1028580013700E4B1A780E4B1A70FA7913469B00B8
:1028680013449B0003F5FA63FB60074B1B681B6866
:10287800FA68DA63044B1B681B68FA681A64143731
:10288800BD465DF8047B70475C0100206D040020A4
:102898006C04002080B483B000AF0D4B1B781A463F
:1028A80013469B0013449B0003F5FA637B60094BB6
:1028B8001B681B687A68DA63064B1B681B687A68B2
:1028C8001A6400BF0C37BD465DF8047B704700BF33
:1028D8006C0400205C01002080B584B000AF7860F3
:1028E8000D4A7B6813600023FB600CE0F86800F079
:1028F80013F90346FB72FB7A002B01D0FB7A06E042
:10290800FB680133FB60FB680C2BEFDD00231846E6
:102918001037BD4680BD00BF8C010020B0B586B021
:1029280002AF03460A46FB711346BB80022000F043
:1029380069FB0C4B00225A800A4AFB7913710A4B37
:10294800FB60BB8800221C461546022300932246E2
:102958002B46F868FEF78CF9F86000BF1037BD46C3
:10296800B0BD00BFB4010020B901002080B584B01B
:1029780000AF0023FB600023BB6000237B609FE067
:102988007B685B005F4A13441946786800F0E4F8F6
:102998000346002B08D15B4A7B6832F913309BB29F
:1029A80003F00F03002B12D001227B6802FA03F315
:1029B8001A46554B1B681343534A1360534B1B78F5
:1029C8000133DAB2514B1A700123FB6075E04D4AAE
:1029D8007B6832F913301B1119B24A4A7B6822F816
:1029E800131001227B6802FA03F3DB431A46464BB5
:1029F8001B681340444A1360454B1B78062B03D0D1
:102A0800434B1B78052B14D13E4A7B6832F91330AF
:102A1800B3F5347F21DB0123BB607B68DAB2394927
:102A28007B6831F913309BB219461046FFF776FFE1
:102A380013E0344A7B6832F91330B3F56C7F0CDB52
:102A48000123BB607B68DAB22E497B6831F9133009
:102A58009BB219461046FFF761FF2D4B1B78062BDA
:102A680003D02B4B1B78052B13D1264A7B6832F9F0
:102A78001330002B21DC0123BB607B68DAB22149CB
:102A88007B6831F913309BB219461046FFF746FFB1
:102A980013E01C4A7B6832F9133013F5A07F0CDC75
:102AA8000123BB607B68DAB216497B6831F91330C1
:102AB8009BB219461046FFF731FF7B6801337B60F4
:102AC8007B680C2B7FF75CAF104B1B78022B06D969
:102AD800104B04225A80022000F094FA05E0BB68EB
:102AE800002B02D1022000F0AFFA084B00221A7026
:102AF800FB68002B14BF01230023DBB218461037F4
:102B0800BD4680BD680100208401002088010020A6
:102B18003C040020B401002080B586B002AF786084
:102B28007B681BB25B001BB243F080031BB2FB81C6
:102B380000233B73074B186807F10C02F9896423DB
:102B48000093012303F00CFB034618461037BD46DB
:102B580080BD00BF8C01002080B586B002AF7860D0
:102B680039607B681BB25B001BB243F080031BB269
:102B7800FB81FB8943F00103FB810F4B186807F1C8
:102B88000802F98905230093022303F0DDFB0346BD
:102B98007B737B7B002B09D13B7A1BB21B021AB2D9
:102BA8007B7A1BB213431AB23B681A807B7B1846A8
:102BB8001037BD4680BD00BF8C01002080B582B0B3
:102BC80000AF78607868FDF787FF40F6FF7140F244
:102BD8000150FDF7C5FF114BFF221A700F4BFF2262
:102BE8005A7002F009F9034603F57A730C4A136028
:102BF80002F002F90346C8330A4A136002F0FCF8EF
:102C0800034603F59C530833074A1360074B002219
:102C18001A7000BF0837BD4680BD00BF9401002070
:102C28009C010020A0010020A401002090010020A8
:102C380080B586B000AF02F0DFF80246594B1B683A
:102C48009A42C0F0AB8007F1100300221A605A6064
:102C580002F0D2F8034603F57A73524A1360002350
:102C6800FB730023BB8107F10C0207F10F03114628
:102C7800184601F079FC4C4B1B785BB21B015AB229
:102C88004A4B1B781B09DBB25BB213435BB2DBB266
:102C98003B74464B1B785BB21B015AB2424B5B88B4
:102CA8001B099BB25BB213435BB2DBB27B743E4B36
:102CB8005B88DBB21B01DBB2BB743D4BD3ED007A02
:102CC800FDEEE77AC7ED017A3B79FB74394B1B6857
:102CD8001846FDF7A7FB4FF00002374BFDF736FD0E
:102CE80002460B4610461946FDF760FE034600EE05
:102CF800103A06F0E3FDF0EE407AFCEEE77AC7ED15
:102D0800017A3B79DBB23B752C4B1B681846FDF703
:102D180089FB4FF00002284BFDF718FD02460B46D1
:102D280010461946FDF742FE034600EE103A06F03B
:102D3800C5FDF0EE407AFCEEE77AC7ED017A3B7903
:102D4800DBB27B751E4B1B681846FDF76BFB4FF01B
:102D58000002194BFDF7FAFC02460B4610461946CD
:102D6800FDF724FE034600EE103A06F0A7FDF0EE4C
:102D7800407AFCEEE77AC7ED017A3B79DBB2BB75A6
:102D8800BB891B099BB2DBB2FB7507F11003082254
:102D9800194640F20250FDF7BFFE00E000BF1837A9
:102DA800BD4680BD9C0100203C0400206C0400202E
:102DB800240400204404002000408F4048040020E0
:102DC8004C04002080B582B000AF02F015F802462E
:102DD800224B1B689A423DD33B4600221A605A6038
:102DE80002F00AF80346C8331C4A13601C4B1B78D0
:102DF8003B701B4B1B781A461A4B33F912301B12C7
:102E08001BB2DBB27B70164B1B781A46154B33F995
:102E18001230DBB2BB70124B1B781A46124B33F9D7
:102E280012301B111BB2DBB2FB703B460422194661
:102E380040F20350FDF770FE094B1B780133DAB2FC
:102E4800074B1A70064B1B780D2B04D1044B00223C
:102E58001A7000E000BF0837BD4680BDA001002001
:102E680090010020D40000206801002080B582B0C5
:102E780000AF78607B681B78002B08D17B68013332
:102E88001B78002B03D1786800F040FF5AE07B687C
:102E98001B78012B08D17B6801331B78002B03D1E9
:102EA800786800F033FF4DE07B681B78022B08D16F
:102EB8007B6801331B78642B03D8786800F026FF01
:102EC80040E07B681B78F02B08D17B6801331B78C6
:102ED800002B03D1786800F019FF33E07B681B787A
:102EE800F12B08D17B6801331B78002B03D178685C
:102EF80000F00CFF26E07B681B78F22B08D17B687A
:102F080001331B78002B03D1786800F0FFFE19E02D
:102F18007B681B78FA2B08D17B6801331B78002B60
:102F280003D1786800F0F2FE0CE07B681B78FF2B79
:102F380008D17B6801331B78002B03D1786800F037
:102F4800E5FEFFE700BF0837BD4680BD80B584B009
:102F580000AF0346B9607A60FB811A4B1B78002BDF
:102F680003D07868FFF782FF28E0FB8940F201521E
:102F7800934223D1BB68022B20D101F03DFF0346C9
:102F880003F59C530833104A1360104B1A787B687A
:102F98001B789A4206D10D4B5A787B6801331B780F
:102FA8009A420BD07B681A78084B1A707B680133F9
:102FB8001A78064B5A707868FFF758FF1037BD46E5
:102FC80080BD00BF38040020A40100209401002027
:102FD80080B483B000AF7860074A7B681360074B02
:102FE80000221A60064B00221A6000BF0C37BD464B
:102FF8005DF8047B704700BFA8010020AC010020E9
:10300800B001002080B582B000AF0346FB800D4BB5
:103018001B88002B04D101F0EFFE0346094A936098
:10302800084B1B881AB2FB88012101FA03F31BB273
:1030380013431BB29AB2034B1A8000BF0837BD4630
:1030480080BD00BFB401002080B483B000AF034648
:10305800FB800A4B1B881AB2FB88012101FA03F393
:103068001BB2DB431BB213401BB29AB2034B1A804C
:1030780000BF0C37BD465DF8047B7047B4010020E3
:1030880080B582B000AF01F05DFE00F053F800F0AB
:1030980065FB00F0A3F800F0D7F800F055F900F050
:1030A800CBFA00F011F900F08DF900F0EFF900F01B
:1030B80053FA00F0F9FC1748FFF70EFC1648FFF723
:1030C800ADF91648FFF77AFD154A16491648FFF775
:1030D80069FB00F0DFFB154A1449144801F070FA47
:1030E80000F05CFF1248FFF773FFFFF7C9F901F022
:1030F80083FE034603F5FA737B6000BF01F07CFE94
:1031080002467B689342F9D8FFF7BAF900F008FD48
:1031180000BFF9E7E801002090020020C00100206C
:10312800D8030020F4020020400300208C03002074
:103138003C02002080B59CB000AF07F1480328226C
:103148000021184606F0B2FB07F1340300221A608A
:103158005A609A60DA601A613B46342200211846A8
:1031680006F0A4FB0123BB644FF48033FB64012306
:10317800BB6500237B6607F14803184603F004FD8E
:103188000346002B01D000F07FFB0F237B63012354
:10319800BB630023FB6300233B6400237B6407F1CC
:1031A80034030021184604F0FDFC0346002B01D02F
:1031B80000F06AFB60233B601023FB6120233B6225
:1031C8003B46184604F0C8FE0346002B01D000F029
:1031D8005BFB00BF7037BD4680BD000080B500AF07
:1031E800174B184A1A60164B02225A60144B0022D9
:1031F8009A60134B0022DA60114B4FF440221A6197
:103208000F4B4FF480125A610D4B00221A760C4B6B
:1032180001225A760A4B00229A76094B0122DA7665
:10322800074B00221A77064B00225A77044801F010
:1032380013FE0346002B01D000F026FB00BF80BD23
:10324800C00100200064004080B500AF1B4B1C4A41
:103258001A601A4B1B4A5A60184B00229A60174B87
:103268000122DA60154B00221A61144B00225A61C0
:10327800124B00229A61114B0022DA610F4B002297
:103288001A620E4802F0DCFE0346002B01D000F063
:10329800FBFA0021094803F0DFFB0346002B01D0AD
:1032A80000F0F2FA0021054803F021FC0346002B48
:1032B80001D000F0E9FA00BF80BD00BFE80100209E
:1032C800005400405B3D300080B500AF1B4B1C4AEA
:1032D8001A601A4B1B4A5A60184B00229A60174B07
:1032E8000122DA60154B00221A61144B00225A6140
:1032F800124B00229A61114B0022DA610F4B002217
:103308001A620E4802F09CFE0346002B01D000F022
:10331800BBFA0021094803F09FFB0346002B01D0AC
:1033280000F0B2FA0021054803F0E1FB0346002B48
:1033380001D000F0A9FA00BF80BD00BF3C02002008
:10334800005800405B3D300080B500AF1B4B1C4A65
:103358001A601A4B4FF482725A60184B00229A6016
:10336800164B4FF4E062DA60144B00221A61134BDB
:1033780000225A61114B4FF400729A610F4B2022C0
:10338800DA610E4B00221A620C4B00225A620B4B78
:1033980000229A62094B0722DA62084B00221A635C
:1033A800064B08225A63054804F066FF0346002BC3
:1033B80001D000F069FA00BF80BD00BF9002002074
:1033C8000030014080B58AB000AF07F11C0300222D
:1033D8001A605A609A603B4600221A605A609A60E6
:1033E800DA601A615A619A61274B4FF080421A607D
:1033F800254B00225A60244B00229A60224B4FF042
:10340800FF32DA60204B00221A611F4B00229A61BA
:103418001D4805F063FB0346002B01D000F034FA89
:103428000023FB6100237B6207F11C031946164841
:1034380006F002F90346002B01D000F025FA6023BC
:103448003B6000237B600023BB6000233B613B465D
:10345800082219460C4805F08DFC0346002B01D0C4
:1034680000F012FA3B460C221946074805F082FC88
:103478000346002B01D000F007FA034801F068FB6F
:1034880000BF2837BD4680BDF402002080B58AB051
:1034980000AF07F11C0300221A605A609A603B468D
:1034A80000221A605A609A60DA601A615A619A6159
:1034B800274B284A1A60264B07225A60244B0022C1
:1034C8009A60234B49F63F42DA60214B00221A6189
:1034D8001F4B00229A611E4805F000FB0346002B93
:1034E80001D000F0D1F90023FB6100237B6207F1D2
:1034F8001C031946164806F09FF80346002B01D016
:1035080000F0C2F960233B6000237B600023BB60AE
:1035180000233B613B46082219460D4805F02AFC6A
:103528000346002B01D000F0AFF93B460C221946A8
:10353800074805F01FFC0346002B01D000F0A4F952
:10354800034801F005FB00BF2837BD4680BD00BF1A
:10355800400300200004004080B58AB000AF07F1A6
:103568001C0300221A605A609A603B4600221A60C7
:103578005A609A60DA601A615A619A612C4B2D4A36
:103588001A602B4B4FF41C725A60294B00229A6028
:10359800274BFF22DA60264B00221A61244B0022B7
:1035A8009A61234805F09AFA0346002B01D000F0EF
:1035B8006BF90023FB6100237B6207F11C031946AA
:1035C8001B4806F039F80346002B01D000F05CF9DF
:1035D80060233B6000237B600023BB6000233B61CA
:1035E8003B4600221946124805F0C4FB0346002B4F
:1035F80001D000F049F93B46042219460C4805F071
:10360800B9FB0346002B01D000F03EF93B460822E7
:103618001946074805F0AEFB0346002B01D000F021
:1036280033F9034801F094FA00BF2837BD4680BD3E
:103638008C0300200008004080B596B000AF07F169
:103648004C0300221A605A609A6007F13003002286
:103658001A605A609A60DA601A615A619A613B1D71
:103668002C220021184606F021F93A4B3A4A1A60F2
:10367800384B00225A60374B00229A60354B4FF680
:10368800FF72DA60334B00221A61324B00225A6112
:10369800304B00229A612F4805F020FA0346002B90
:1036A80001D000F0F1F80023FB6400237B6507F1EB
:1036B8004C031946274805F0BFFF0346002B01D0ED
:1036C80000F0E2F860233B6300237B630023BB63C5
:1036D8000023FB6300233B6400237B640023BB645B
:1036E80007F13003002219461A4805F043FB034648
:1036F800002B01D000F0C8F807F130030422194666
:10370800144805F037FB0346002B01D000F0BCF845
:1037180000237B600023BB600023FB6000233B6128
:1037280000237B614FF40053BB610023FB6100233E
:10373800FB623B1D1946074805F0F2FF0346002BC4
:1037480001D000F0A1F8034801F002FA00BF583791
:10375800BD4680BDD80300200040014080B58AB036
:1037680000AF07F1140300221A605A609A60DA6009
:103778001A61424B5B69414A43F4002353613F4B52
:103788005B6903F400233B613B693C4B5B693B4A43
:1037980043F480035361394B5B6903F48003FB6096
:1037A800FB68364B5B69354A43F400335361334B4E
:1037B8005B6903F40033BB60BB68304B5B692F4A1D
:1037C80043F4802353612D4B5B6903F480237B60B2
:1037D8007B6800224FF488714FF0904002F018FC8B
:1037E80000223021264802F013FC4FF460437B612D
:1037F8000323BB610023FB6107F114031946214829
:1038080002F08CFA0F237B610323BB610023FB6169
:1038180007F1140319464FF0904002F07FFA4FF475
:1038280088737B610123BB610023FB6103233B6237
:1038380007F1140319464FF0904002F06FFA43F273
:1038480004037B610323BB610023FB6107F11403BD
:1038580019460B4802F062FA30237B610123BB61F1
:103868000023FB6100233B6207F114031946044857
:1038780002F054FA00BF2837BD4680BD0010024050
:10388800000400480008004880B400AF72B600BFCA
:1038980000BFFDE780B400AF074B4FF000021A608D
:1038A800064B00221A60064B01221A6000BFBD4673
:1038B8005DF8047B704700BF240400202C0400201E
:1038C8002804002080B584B000AF01F095FAF860B4
:1038D800334B1B68B3F57A7F17DB324AFB681360FA
:1038E800314B1B68002B0CD1304B1B68304A1360DE
:1038F8002B4B1B6807EE903AF8EEE77A2D4BC3ED99
:10390800007A294B01221A6002E0274B00221A6034
:10391800244B1B68FA68D31A274A934203D8214BD1
:103928001B68002B13D10023FB7000233B803A4611
:10393800FB1C1146184600F017FE3B88184600F09D
:1039480041F8F0EE407A194BC3ED007A23E0144BAE
:103958001B6807EE903AB8EEE77A164BD3ED007A7B
:1039680077EE677AC7ED027A97ED027ADFED136A90
:10397800C7EE267A9FED127A67EE877AC7ED017A4D
:103988000B4B93ED007AD7ED017A77EE277A074B48
:10399800C3ED007A00BF00BF1037BD4680BD00BF31
:1039A8004C0400202C0400202804002024040020BB
:1039B80030040020340400209F8601000000E14606
:1039C8000000C84280B48BB000AF0346FB800023E0
:1039D8007B620B233B6202E07B6A01337B627A6A7B
:1039E8003B6A9A4206D22F4A7B6A32F83330FA8809
:1039F8009A42F1D27B6A002B02D12A4B5B6848E0DD
:103A08007A6A3B6A9A4207D13B6A013B254ADB0046
:103A1800134404331B683CE07B6A013B214A32F8BB
:103A28003330FB831F4A7B6A32F83330BB837B6AAF
:103A3800013B1C4ADB00134404331B68BB61194A71
:103A48007B6ADB00134404331B687B6197ED057ABE
:103A5800D7ED067A77EE676ABA8BFB8BD31A07EE37
:103A6800903AB8EEE77AC6EE877AC7ED047AFA8814
:103A7800FB8BD31A07EE903AB8EEE77AD7ED047AC3
:103A880067EE277A97ED067A77EE277AC7ED037AFD
:103A9800FB6807EE903AB0EE670A2C37BD465DF832
:103AA800047B70470400002080B400AF134B002251
:103AB8001A70124B00225A70104B00225A80104B79
:103AC80000221A600E4B1B680E4A13600D4B1B68D0
:103AD8000D4A13600C4B1B680C4A13600B4B1B6898
:103AE8000B4A13600B4B00221A700B4B00221A7002
:103AF80000BFBD465DF8047B704700BF3C04002052
:103B08006004002054040020680400205C040020A5
:103B18005804002038040020390400200000000068
:103B280080B500AF704BD3ED087A9FED707AF4EE54
:103B3800C77AF1EE10FA1ADD6B4B1B6A1846FCF7D0
:103B480083FC63A3D3E90023FCF71EFB02460B4664
:103B58001046194660A3D3E90023FCF7CDFC0246C2
:103B68000B4610461946FCF7D9FE034600E0002331
:103B78005F4A13605C4BD3ED097A9FED5E7AF4EEF1
:103B8800C77AF1EE10FACCBF01230023DAB25A4B00
:103B98001A70554B9B6A1846FCF756FC50A3D3E99C
:103BA8000023FCF7A9FC02460B4610461946FCF711
:103BB800B5FE0346514A13604B4BDB6A1846FCF7C7
:103BC80043FC47A3D3E90023FCF796FC02460B46C7
:103BD80010461946FCF7A2FE0346494A136001F055
:103BE8000BF90246474B1B689A4206D9464B0722F7
:103BF8005A70454B5A78444B1A70FFF719F8FFF77B
:103C0800E1F800F0E7F900F007F900F073F9FEF7C2
:103C1800ADFE00F00FFDFFF755FE3B4B1B78072B61
:103C28004AD801A252F823F0513C00085F3C000832
:103C38006D3C00087B3C0008893C0008973C000864
:103C4800A53C0008B33C000800F04CFB03461A46AC
:103C58002D4B1A7030E000F061FB03461A462A4BE0
:103C68001A7029E000F070FB03461A46264B1A70BA
:103C780022E000F07FFB03461A46234B1A701BE034
:103C880000F08EFB03461A461F4B1A7014E000F032
:103C98009DFB03461A461C4B1A700DE000F0AAFB68
:103CA80003461A46184B1A7006E000F0BBFB0346A1
:103CB8001A46154B1A7000BF134B1B78184600F0B4
:103CC800C5FB114B1A78104B5A7000BF80BD00BF5E
:103CD80000000000007EA3400000000000C0724009
:103CE800E17A14AE47612E40D400002000F01B4555
:103CF8004C04002000001645500400204804002011
:103D080044040020A40100203C04002080B582B0B7
:103D180000AF78603D4B1B78002B0DD03C4B1B78D7
:103D2800022B03D03A4B1B78032B05D17B68013358
:103D38001B781846FEF770FD7B681B78FF2B50D068
:103D4800FF2B5EDCF12B53D0F12B5ADCF02B40D04B
:103D5800F02B56DC022B2BD0022B52DC002B02D08E
:103D6800012B0BD04DE02A4B1B78002B42D0284B5F
:103D780004225A70FF20FEF74FFD3BE0244B5B788E
:103D8800002B03D0224B5B78042B06D1204B012259
:103D98005A700020FEF740FD2EE01D4B5B78032B88
:103DA8002AD11B4B02225A700020FEF735FD23E072
:103DB800174B1B78022B03D0154B1B78032B1DD1F7
:103DC8007B6801331A78134B1A70114B03225A700F
:103DD80014E00F4B1B78002B12D10D4B05225A70A3
:103DE8000EE00B4B04221A70094B07225A7008E0A8
:103DF80000BF06E000BF04E000BF02E000BF00E033
:103E080000BF00BF0837BD4680BD00BF3804002092
:103E18003C0400206D04002080B500AF324B1B78B5
:103E2800012B0BD0304B5B78012B07D100F0E4FF5E
:103E3800034603F5FA532D4A136010E02A4B1B780A
:103E4800012B0CD100F0D8FF0246284B1B689A4280
:103E580005D9254B02225A70244B00221A60224BA6
:103E68001B78052B0BD0204B5B78052B07D100F076
:103E7800C3FF034603F5FA531C4A136010E01A4BBC
:103E88001B78052B0CD100F0B7FF0246174B1B68B7
:103E98009A4205D9144B06225A70144B00221A6014
:103EA800114B1B78042B0BD00F4B5B78042B07D1DD
:103EB80000F0A2FF034603F5FA530D4A136010E021
:103EC800094B1B78042B0CD100F096FF0246084BD7
:103ED8001B689A4205D9044B00225A70044B0022F1
:103EE8001A6000BF80BD00BF3C04002058040020B9
:103EF8005C04002080B500AF254B1A78254B1B7851
:103F08009A4243D0224B1B78642B03D8214B1B7851
:103F1800642B0AD9FF20FEF77FFC1E4B00221A7083
:103F28001C4B1A781A4B1A7031E000F065FF0246F4
:103F3800194B1B689A422AD9154B1A78154B1B78CE
:103F48009A420ED2124B1B780533DAB2104B1A7014
:103F5800FEF7A0FC00F050FF03460F330E4A136033
:103F680015E00B4B1A780B4B1B789A420FD9084B6C
:103F78001B78053BDAB2064B1A70FEF78BFC00F093
:103F88003BFF03460F33044A136000E000BF80BDC7
:103F98006C0400206D0400206404002080B500AF8C
:103FA8000A4B1B7883F00103DBB2002B0CD1642091
:103FB800FEF732FC064B03225A70054B5A78044B25
:103FC8001A70FEF735FEFCE700BF80BD38040020FC
:103FD8003C04002080B500AF774B1B78002B40F0E5
:103FE800E880764B1B78002B40F0E380744B1B88ED
:103FF80003F00103002B0BD1714B1B8803F0020364
:10400800002B05D16E4B1B8803F01003002B01D049
:10401800012300E0002303F00103D9B2694A1379B0
:1040280061F382031371664B1B8803F00403002BB2
:1040380011D1634B1B8803F00803002B0BD1604B95
:104048001B8803F02003002B05D15F4B1B6847F248
:104058002F52934201DC012300E0002303F0010307
:10406800D9B2584A137961F345131371544B1B881D
:10407800DB1103F00103D9B2524A137961F300034B
:1040880013714F4B1B8803F48073002B0BD14C4BDF
:104098001B8803F48063002B05D1494B1B8803F46C
:1040A8000073002B01D0012300E0002303F001037B
:1040B800D9B2444A137961F341031371434B1B7816
:1040C80083F00103D9B23F4A137961F304131371E2
:1040D8003D4B1B6840F2E7329342D4BF01230023D3
:1040E800D9B2384A137961F386131371354B1B79AA
:1040F80003F00803DBB2002B30D1324B1B7903F0FD
:104108001003DBB2002B29D12E4B1B7923F07F0340
:10411800DBB2002B22D12B4B1B7903F00403DBB25B
:10412800002B1BD1274B1B7903F02003DBB2002B9C
:1041380014D1244B1B7903F04003DBB2002B0DD1C3
:10414800204B1B7903F00203DBB2002B06D11D4B79
:104158001B7903F00103DBB2002B19D0194B1B7834
:10416800002B06D0174B1B78072B02D0154B0422C7
:104178001A70144B07225A70FF20FEF74DFB00F00F
:104188003BFE034603F51C531033114A13600DE040
:104198000C4B1B78072B09D100F02EFE02460C4B66
:1041A8001B689A4202D9074B00225A7000F012F895
:1041B80000E000BF80BD00BF3804002039040020A3
:1041C800B40100203C0400204404002050040020D6
:1041D8005404002080B400AF414B00225A80404B69
:1041E8005B883F4A1279C2F30002D2B213439AB2F3
:1041F8003B4B5A803A4B5B881AB2394B1B79C3F355
:104208004003DBB21BB25B001BB213431BB29AB272
:10421800334B5A80324B5B881AB2314B1B79C3F34C
:104228008003DBB21BB29B001BB213431BB29AB2D2
:104238002B4B5A802A4B5B881AB2294B1B79C3F344
:10424800C003DBB21BB2DB001BB213431BB29AB232
:10425800234B5A80224B5B881AB2214B1B79C3F33C
:104268000013DBB21BB21B011BB213431BB29AB281
:104278001B4B5A801A4B5B881AB2194B1B79C3F334
:104288004013DBB21BB25B011BB213431BB29AB2E1
:10429800134B5A80124B5B881AB2114B1B79C3F32C
:1042A8008013DBB21BB29B011BB213431BB29AB241
:1042B8000B4B5A800A4B5B881AB2094B1B79C3F324
:1042C800C013DBB21BB2DB011BB213431BB29AB2A1
:1042D800034B5A8000BFBD465DF8047B704700BFA2
:1042E8003C04002080B400AF0B4B5B78072B0AD04E
:1042F800072B0ADC012B02D0052B02D005E0012395
:1043080004E0052302E0072300E000231846BD4629
:104318005DF8047B704700BF3C04002080B400AF08
:10432800084B5B78002B02D0022B02D003E0042359
:1043380002E0022300E001231846BD465DF8047B35
:10434800704700BF3C04002080B400AF084B5B7886
:10435800032B02D0042B02D003E0032302E0042342
:1043680000E002231846BD465DF8047B704700BF95
:104378003C04002080B400AF084B5B78022B02D0CD
:10438800042B02D003E0022302E0042300E003230D
:104398001846BD465DF8047B704700BF3C0400200A
:1043A80080B400AF084B5B78002B02D0072B02D0FB
:1043B80003E0002302E0072300E004231846BD467B
:1043C8005DF8047B704700BF3C04002080B400AF58
:1043D800074B5B78042B03D0062B03D1062302E09E
:1043E800042300E005231846BD465DF8047B7047AA
:1043F8003C04002080B400AF084B5B78042B04D148
:10440800074B01221A70042303E0054B02221A709D
:1044180006231846BD465DF8047B70473C0400201F
:104428004F01002080B400AF074B5B78002B03D00E
:10443800042B03D1042302E0002300E007231846DD
:10444800BD465DF8047B70473C04002080B582B00F
:1044580000AF0346FB71314B1B78072B5AD801A2DA
:1044680052F823F08D4400089F440008B144000826
:10447800C3440008D5440008E7440008F94400088C
:104488000B4500080021002000F04AF80021012017
:1044980000F046F83EE00021002000F041F801213C
:1044A800012000F03DF835E00121002000F038F847
:1044B8000021012000F034F82CE00121002000F058
:1044C8002FF80021012000F02BF823E00021002024
:1044D80000F026F80121012000F022F81AE000215E
:1044E800002000F01DF80121012000F019F811E06A
:1044F8000121002000F014F80021012000F010F83C
:1045080008E00021002000F00BF80021012000F055
:1045180007F800BF00BF0837BD4680BD3C04002037
:1045280080B584B000AF03460A46FB711346BB71E1
:10453800BB79FB73FB79002B02D0012B07D00DE070
:10454800FB7B1A461021074801F062FD06E0FB7B61
:104558001A462021034801F05BFD00BF00BF103759
:10456800BD4680BD0004004880B485B000AF7860C7
:1045780039600023FB6016E0104AFB6832F91330FB
:104588001A463B681B889A420ADDFB68DAB27B68E8
:104598001A700A4AFB6832F913309AB23B681A80DB
:1045A800FB680133FB60FB680C2BE5DD00BF00BF37
:1045B8001437BD465DF8047B704700BF68010020D2
:1045C80080B584B000AFF860B9607A60144AFB68BF
:1045D8001360144ABB681360134A7B681360134B5B
:1045E80000221A60124B00221A700D4B1B68002122
:1045F800184604F0CBFA0B4B1B680421184604F04C
:10460800C5FA094B1B680821184604F0BFFAFF22B7
:10461800FF21FF2000F0D0F800BF1037BD4680BD55
:104628007004002074040020780400207C0400201A
:104638008004002080B500AF344B1B78072B03D1D2
:10464800012000F069F860E000F0D6FB0246304B2C
:104658001B689A4258D32F4B1B78002B17D02B4B33
:104668001B78002B06D100F0C7FB0346C833284A45
:10467800136005E000F0C0FB03463233244A1360A0
:10468800244B00221A70002000F046F83DE01F4B32
:104698001B78002B07D100F0AFFB034603F5FA6344
:1046A8001B4A136006E000F0A7FB034603F5FA7304
:1046B800174A1360174B01221A70144B1B78072BEB
:1046C80023D801A252F823F0F1460008F946000861
:1046D8000147000801470008F9460008F9460008A4
:1046E8000147000809470008022000F015F80CE00F
:1046F800042000F011F808E0052000F00DF804E0AF
:10470800012000F009F800E000BF80BD3C04002053
:104718007C0400208004002080B582B000AF0346EE
:10472800FB71FB79072B43D801A252F823F000BF95
:10473800AD47000859470008654700087147000859
:104748007D4700088947000895470008A1470008E9
:10475800FF22FF21002000F02FF829E0FF2200218E
:10476800FF2000F029F823E00022FF21FF2000F0BD
:1047780023F81DE0FF220021002000F01DF817E0BB
:104788000022FF21002000F017F811E0002200218C
:10479800FF2000F011F80BE000220021002000F0BB
:1047A8000BF805E0FF22FF21FF2000F005F800BF0D
:1047B80000BF0837BD4680BD80B483B000AF034654
:1047C800FB710B46BB7113467B710A4B1B681B6858
:1047D800FA795A63084B1B681B68BA799A63074BC6
:1047E8001B681B687A79DA6300BF0C37BD465DF831
:1047F800047B7047700400207404002078040020B3
:1048080080B483B000AF0F4B9B690E4A43F001039D
:1048180093610C4B9B6903F001037B607B68094B38
:10482800DB69084A43F08053D361064BDB6903F028
:1048380080533B603B6800BF0C37BD465DF8047B86
:10484800704700BF0010024080B58AB000AF7860A2
:1048580007F1140300221A605A609A60DA601A613C
:104868007B681B68204A934239D1204BDB691F4A79
:1048780043F00073D3611D4BDB6903F000733B61A8
:104888003B691A4B5B69194A43F400335361174B70
:104898005B6903F40033FB60FB684FF4C0537B6132
:1048A8000223BB610023FB6103233B6209237B6274
:1048B80007F1140319464FF0904001F02FFA002237
:1048C8000021142001F0F3F9142001F00CFA002261
:1048D8000021152001F0EBF9152001F004FA00BFC2
:1048E8002837BD4680BD00BF00640040001002406C
:1048F80080B58CB000AF786007F11C0300221A6005
:104908005A609A60DA601A617B681B683E4A934273
:1049180047D13E4B5B693D4A43F4003353613B4BFF
:104928005B6903F40033BB61BB69384B5B69374A89
:1049380043F480235361354B5B6903F480237B6127
:104948007B694FF40043FB6112233B6200237B62C7
:104958000323BB620423FB6207F11C0319464FF0D3
:10496800904001F0DBF94FF40073FB6112233B62C6
:1049780000237B620323BB620423FB6207F11C0351
:104988001946234801F0CAF9204BDB691F4A43F452
:104998000013D3611D4BDB6903F400133B613B69D2
:1049A8002EE07B681B681B4A934229D1174B5B6931
:1049B800164A43F400335361144B5B6903F4003324
:1049C800FB60FB684FF4C063FB6112233B6200236A
:1049D8007B620323BB620423FB6207F11C031946B5
:1049E8004FF0904001F09AF9084BDB69074A43F40D
:1049F8008003D361054BDB6903F48003BB60BB68AC
:104A080000BF3037BD4680BD005400400010024052
:104A1800000400480058004080B58AB000AF7860B4
:104A280007F1140300221A605A609A60DA601A616A
:104A38007B681B68174A934228D1174B9B69164A13
:104A480043F480539361144B9B6903F480533B6197
:104A58003B69114B5B69104A43F4003353610E4BB9
:104A68005B6903F40033FB60FB68E0237B6102238E
:104A7800BB610023FB6103233B6205237B6207F1D3
:104A8800140319464FF0904001F048F900BF283749
:104A9800BD4680BD003001400010024080B487B0A0
:104AA80000AF78607B681B68B3F1804F0CD1244B52
:104AB800DB69234A43F00103D361214BDB6903F02F
:104AC80001037B617B6934E07B681B681D4A934264
:104AD8000CD11B4BDB691A4A43F00203D361184B14
:104AE800DB6903F002033B613B6922E07B681B68DA
:104AF800154A93420CD1124BDB69114A43F0040367
:104B0800D3610F4BDB6903F00403FB60FB6810E023
:104B18007B681B680D4A93420BD1094B9B69084A75
:104B280043F480339361064B9B6903F48033BB6085
:104B3800BB6800BF1C37BD465DF8047B704700BFEB
:104B480000100240000400400008004000400140FE
:104B580080B58CB000AF786007F11C0300221A60A2
:104B68005A609A60DA601A617B681B68B3F1804FFB
:104B78001DD1444B5B69434A43F480235361414B45
:104B88005B6903F48023BB61BB694FF44063FB613D
:104B980002233B6200237B620023BB620123FB628A
:104BA80007F11C031946384801F0B8F866E07B683D
:104BB8001B68364A93421CD1324B5B69314A43F435
:104BC800802353612F4B5B6903F480237B617B69EE
:104BD8000323FB6102233B6200237B620023BB6249
:104BE8000223FB6207F11C031946274801F096F8D7
:104BF80044E07B681B68264A93421DD1214B5B69C0
:104C0800204A43F4802353611E4B5B6903F48023DD
:104C18003B613B694FF4E073FB6102233B62022373
:104C28007B620023BB620223FB6207F11C03194667
:104C3800154801F073F821E07B681B68154A934218
:104C48001CD1104B5B690F4A43F4802353610D4B11
:104C58005B6903F48023FB60FB684FF44043FB610E
:104C680002233B6200237B620023BB620123FB62B9
:104C780007F11C031946044801F050F800BF30370B
:104C8800BD4680BD001002400004004800040040FA
:104C9800000800400040014080B400AF00BFFDE7BD
:104CA80080B400AF00BFFDE780B400AF00BFFDE7F0
:104CB80080B400AF00BFFDE780B400AF00BFFDE7E0
:104CC80080B400AF00BFBD465DF8047B704780B478
:104CD80000AF00BFBD465DF8047B704780B400AFED
:104CE80000BFBD465DF8047B704780B500AF00F09B
:104CF8006FF800BF80BD000080B500AF024800F02B
:104D0800CCFC00BF80BD00BFC001002080B500AF53
:104D1800024800F0C2FC00BF80BD00BFC0010020F7
:104D280080B400AF064BD3F88830054A43F47003CB
:104D3800C2F8883000BFBD465DF8047B704700BFED
:104D480000ED00E080B500AF084B1B68074A43F050
:104D580010031360032000F09FFF0F2000F008F8F5
:104D6800FFF74EFD0023184680BD00BF002002401B
:104D780080B582B000AF7860124B1A68124B1B786E
:104D880019464FF47A73B3FBF1F3B2FBF3F3184609
:104D980000F0B7FF0346002B01D001230EE07B682B
:104DA8000F2B0AD8002279684FF0FF3000F07FFF00
:104DB800064A7B681360002300E001231846083781
:104DC800BD4680BD5C00002064000020600000201B
:104DD80080B400AF064B1B781A46064B1B68134479
:104DE800044A136000BFBD465DF8047B704700BFEE
:104DF800640000208404002080B400AF034B1B68CB
:104E08001846BD465DF8047B704700BF8404002047
:104E180080B584B000AF7860FFF7EEFFB8607B68BC
:104E2800FB60FB68B3F1FF3F05D00A4B1B781A46BD
:104E3800FB681344FB6000BFFFF7DEFF0246BB6858
:104E4800D31AFA689A42F7D800BF00BF1037BD4698
:104E580080BD00BF6400002080B584B000AF7860DA
:104E68007B68002B01D10123EDE07B6893F82030AB
:104E7800DBB2002B02D17868FFF7E6FC7B681B6881
:104E88001A687B681B6842F001021A60FFF7B4FFDA
:104E9800F86012E0FFF7B0FF0246FB68D31A0A2B4E
:104EA8000BD97B685B6A43F400327B685A627B6883
:104EB800052283F820200123C5E07B681B685B6816
:104EC80003F00103002BE5D07B681B681A687B6838
:104ED8001B6822F002021A60FFF78EFFF86012E0EA
:104EE800FFF78AFF0246FB68D31A0A2B0BD97B68A7
:104EF8005B6A43F400327B685A627B68052283F858
:104F0800202001239FE07B681B685B6803F0020395
:104F1800002BE5D17B681B7E012B08D17B681B68C1
:104F28001A687B681B6842F080021A6007E07B6899
:104F38001B681A687B681B6822F080021A607B680D
:104F48005B7E012B08D17B681B681A687B681B682D
:104F580042F040021A6007E07B681B681A687B68A9
:104F68001B6822F040021A607B689B7E012B08D1E7
:104F78007B681B681A687B681B6842F020021A600D
:104F880007E07B681B681A687B681B6822F02002B0
:104F98001A607B68DB7E012B08D17B681B681A6866
:104FA8007B681B6822F010021A6007E07B681B68A8
:104FB8001A687B681B6842F010021A607B681B7FC6
:104FC800012B08D17B681B681A687B681B6842F054
:104FD80008021A6007E07B681B681A687B681B6810
:104FE80022F008021A607B685B7F012B08D17B687E
:104FF8001B681A687B681B6842F004021A6007E0A5
:105008007B681B681A687B681B6822F004021A60B8
:105018007B689A687B68DB681A437B681B691A435C
:105028007B685B6942EA03017B685B685A1E7B68A0
:105038001B680A43DA617B6800225A627B68012296
:1050480083F82020002318461037BD4680BD80B461
:1050580087B000AF786039607B681B687B617B68CC
:1050680093F82030FB74FB7C012B03D0FB7C022BD4
:1050780040F0AA807B69D3F8003243F001027B69D3
:10508800C3F800223B685B6903F01F03012202FAA0
:1050980003F3FB607B69D3F81C22FB68DB431A40EF
:1050A8007B69C3F81C223B68DB69002B23D17B6931
:1050B800D3F80C22FB68DB431A407B69C3F80C2247
:1050C8003B68DB6819043B685B689BB23A685269C5
:1050D80019437B69483243F832103B689B681904CE
:1050E8003B681B689AB23B685B690A437969483335
:1050F800DB000B445A603B68DB69012B22D17B69DA
:10510800D3F80C22FB681A437B69C3F80C223B686E
:105118001B6819043B685B689BB23A68526919437B
:105128007B69483243F832103B689B6819043B6836
:10513800DB689AB23B685B690A4379694833DB00EC
:105148000B445A603B689B69002B09D17B69D3F8F3
:105158000422FB68DB431A407B69C3F8042207E09A
:105168007B69D3F80422FB681A437B69C3F80422DD
:105178003B681B69002B09D17B69D3F81422FB68B3
:10518800DB431A407B69C3F8142207E07B69D3F834
:105198001422FB681A437B69C3F814223B681B6A14
:1051A800012B07D17B69D3F81C22FB681A437B6962
:1051B800C3F81C227B69D3F8003223F001027B6913
:1051C800C3F80022002306E07B685B6A43F4802270
:1051D8007B685A62012318461C37BD465DF8047B7C
:1051E800704780B584B000AF78607B6893F8203052
:1051F800DBB2012B2ED17B68022283F820207B684A
:105208001B681A687B681B6822F001021A60FFF7A6
:10521800F3FDF86012E0FFF7EFFD0246FB68D31AD2
:105228000A2B0BD97B685B6A43F400327B685A62AD
:105238007B68052283F82020012312E07B681B6825
:105248005B6803F00103002BE5D17B6800225A62FA
:10525800002306E07B685B6A43F400227B685A629D
:10526800012318461037BD4680BD80B489B000AF11
:10527800F860B9607A603B60FB6893F82030FB7790
:10528800FB681B689B68BB61FB7F012B03D0FB7F1E
:10529800022B40F0AD80BB6903F08063002B0AD17C
:1052A800BB6903F00063002B05D1BB6903F0805391
:1052B800002B00F09580BB691B0E03F003037B6194
:1052C80001227B699A403B681A60BB689B68002B87
:1052D8000DD1BB681B685A05BB68DB68F9680968AB
:1052E8001A437B6918331B010B441A600FE0BB6833
:1052F8005B68DA00BB689B681A43BB68DB68F968BF
:1053080009681A437B6918331B010B441A60FB6850
:105318001968BB681A697B6918331B010B4404338D
:105328001A60BB681B7D012B11D1FB681A687B6969
:1053380018331B01134404331B68FA68116843F4DB
:1053480080727B6918331B010B4404331A607B6835
:1053580007331B781A067B6806331B781B041A432D
:105368007B6805331B781B0213437A680432127872
:105378001046FA68116843EA00027B691B010B4476
:1053880003F5C6731A607B6803331B781A067B68BB
:1053980002331B781B041A437B6801331B781B02FA
:1053A80013437A6812781046FA68116843EA0002D3
:1053B8007B691B010B4403F5C4731A60FB681A6808
:1053C8007B6918331B0113441B68FA68116843F0A2
:1053D80001027B6918331B010B441A6000230EE09D
:1053E800FB685B6A43F40012FB685A62012306E01B
:1053F800FB685B6A43F48022FB685A620123184603
:105408002437BD465DF8047B704780B487B000AF91
:10541800F860B9607A603B60FB6893F82030FB75F0
:10542800FB7D012B03D0FB7D022B40F00381BB6881
:10543800002B0ED1FB681B68DB6803F00303002B0D
:1054480016D1FB685B6A43F40012FB685A620123B9
:10545800F7E0FB681B681B6903F00303002B07D107
:10546800FB685B6A43F40012FB685A620123E8E0B8
:10547800FB681A68BB681B331B0113441B6803F0E5
:1054880004027B689A607B689B68002B0CD1FB68E0
:105498001A68BB681B331B0113441B685B0DC3F3FD
:1054A8000A027B681A600BE0FB681A68BB681B334A
:1054B8001B0113441B68DB0823F060427B685A60B9
:1054C800FB681A68BB681B331B0113441B6803F095
:1054D80002027B68DA60FB681A68BB681B331B0131
:1054E800134404331B6803F00803002B03D07B68C4
:1054F80008221A610BE0FB681A68BB681B331B01A2
:10550800134404331B6803F00F027B681A61FB68BD
:105518001A68BB681B331B01134404331B681B0A3E
:10552800DAB27B689A61FB681A68BB681B331B0197
:10553800134404331B681B0C9AB27B685A61FB68DE
:105548001A68BB681B01134403F5DC731B68DAB2E5
:105558003B681A70FB681A68BB681B01134403F5A3
:10556800DC731B681A0A3B680133D2B21A70FB68F5
:105578001A68BB681B01134403F5DC731B681A0C1B
:105588003B680233D2B21A70FB681A68BB681B0109
:10559800134403F5DC731B681A0E3B680333D2B25D
:1055A8001A70FB681A68BB681B01134403F5DE73A5
:1055B8001A683B680433D2B21A70FB681A68BB6871
:1055C8001B01134403F5DE731B681A0A3B68053395
:1055D800D2B21A70FB681A68BB681B01134403F542
:1055E800DE731B681A0C3B680633D2B21A70FB686C
:1055F8001A68BB681B01134403F5DE731B681A0E97
:105608003B680733D2B21A70BB68002B08D1FB681D
:105618001B68DA68FB681B6842F02002DA6007E062
:10562800FB681B681A69FB681B6842F020021A6154
:10563800002306E0FB685B6A43F48022FB685A6239
:10564800012318461C37BD465DF8047B704780B4BB
:1056580085B000AF786039607B6893F82030FB73C1
:10566800FB7B012B02D0FB7B022B09D17B681B68DB
:1056780059697B681B683A680A435A61002306E047
:105688007B685B6A43F480227B685A620123184670
:105698001437BD465DF8047B704780B58AB000AF0B
:1056A800786000237B627B681B685B693B627B6870
:1056B8001B685B68FB617B681B689B68BB617B68D8
:1056C8001B68DB687B617B681B681B693B617B68C7
:1056D8001B689B69FB603B6A03F00103002B7CD0CD
:1056E800BB6903F00103002B23D07B681B680122F0
:1056F8009A60BB6903F00203002B03D0786800F0BE
:1057080083F916E0BB6903F00403002B04D07B6A1D
:1057180043F400637B620CE0BB6903F00803002BD1
:1057280004D07B6A43F480537B6202E0786800F01F
:1057380089F9BB6903F48073002B24D07B681B684C
:105748004FF480729A60BB6903F40073002B03D096
:10575800786800F063F916E0BB6903F48063002BF6
:1057680004D07B6A43F400537B620CE0BB6903F40A
:105778000063002B04D07B6A43F480437B6202E021
:10578800786800F069F9BB6903F48033002B24D0F2
:105798007B681B684FF480329A60BB6903F400335E
:1057A800002B03D0786800F043F916E0BB6903F4D6
:1057B8008023002B04D07B6A43F400437B620CE017
:1057C800BB6903F40023002B04D07B6A43F48033C5
:1057D8007B6202E0786800F049F93B6A03F008034D
:1057E800002B0CD07B6903F01003002B07D07B6AD9
:1057F80043F400737B627B681B681022DA603B6AA3
:1058080003F00403002B0BD07B6903F00803002B83
:1058180006D07B681B680822DA60786800F030F9E7
:105828003B6A03F00203002B09D07B681B68DB6826
:1058380003F00303002B02D07868FBF7EDF93B6A0D
:1058480003F04003002B0CD03B6903F01003002B3E
:1058580007D07B6A43F480637B627B681B681022F5
:105868001A613B6A03F02003002B0BD03B6903F05D
:105878000803002B06D07B681B6808221A61786829
:1058880000F012F93B6A03F01003002B09D07B6883
:105898001B681B6903F00303002B02D0786800F033
:1058A800F9F83B6A03F40033002B0BD0FB6903F0D3
:1058B8001003002B06D07B681B6810225A6078689A
:1058C80000F0FCF83B6A03F48033002B0BD0FB6933
:1058D80003F00803002B06D07B681B6808225A6077
:1058E800786800F0F5F83B6A03F40043002B7BD09E
:1058F800FB6903F00403002B72D03B6A03F4807346
:10590800002B08D0FB6803F00103002B03D07B6A4F
:1059180043F001037B623B6A03F40073002B08D059
:10592800FB6803F00203002B03D07B6A43F00203F9
:105938007B623B6A03F48063002B08D0FB6803F0AA
:105948000403002B03D07B6A43F004037B623B6AA9
:1059580003F40063002B43D0FB6803F07003002BB3
:105968003ED0FB6803F07003602B2BD0602B2ED841
:10597800502B22D0502B2AD8402B19D0402B26D878
:10598800302B10D0302B22D8102B02D0202B05D052
:105998001DE07B6A43F008037B6219E07B6A43F0F1
:1059A80010037B6214E07B6A43F020037B620FE004
:1059B8007B6A43F040037B620AE07B6A43F0800322
:1059C8007B6205E07B6A43F480737B6200E000BF82
:1059D8007B681B689A697B681B6822F070029A6171
:1059E8007B681B6804225A607B6A002B08D07B689E
:1059F8005A6A7B6A1A437B685A62786800F072F8C0
:105A080000BF2837BD4680BD80B483B000AF786042
:105A180000BF0C37BD465DF8047B704780B483B087
:105A280000AF786000BF0C37BD465DF8047B704757
:105A380080B483B000AF786000BF0C37BD465DF816
:105A4800047B704780B483B000AF786000BF0C3728
:105A5800BD465DF8047B704780B483B000AF7860C2
:105A680000BF0C37BD465DF8047B704780B483B037
:105A780000AF786000BF0C37BD465DF8047B704707
:105A880080B483B000AF786000BF0C37BD465DF8C6
:105A9800047B704780B483B000AF786000BF0C37D8
:105AA800BD465DF8047B704780B483B000AF786072
:105AB80000BF0C37BD465DF8047B704780B483B0E7
:105AC80000AF786000BF0C37BD465DF8047B7047B7
:105AD80080B483B000AF786000BF0C37BD465DF876
:105AE800047B704780B483B000AF786000BF0C3788
:105AF800BD465DF8047B704780B485B000AF786020
:105B08007B6803F00703FB600C4BDB68BB60BA687B
:105B18004FF6FF031340BB60FB681A02BB681343D0
:105B280043F0BF6343F40033BB60044ABB68D360EF
:105B380000BF1437BD465DF8047B704700ED00E0F8
:105B480080B400AF044BDB681B0A03F00703184658
:105B5800BD465DF8047B704700ED00E080B483B07B
:105B680000AF0346FB7197F90730002B0BDBFB797D
:105B780003F01F02074997F907305B09012000FA73
:105B880002F241F8232000BF0C37BD465DF8047BC4
:105B9800704700BF00E100E080B483B000AF034667
:105BA8003960FB7197F90730002B0ADB3B68DAB2E2
:105BB8000C4997F907301201D2B20B4483F800233D
:105BC8000AE03B68DAB20849FB7903F00F03043BAB
:105BD8001201D2B20B441A7600BF0C37BD465DF8ED
:105BE800047B704700E100E000ED00E080B489B07C
:105BF80000AFF860B9607A60FB6803F00703FB61E7
:105C0800FB69C3F10703042B28BF0423BB61FB69AD
:105C18000433062B02D9FB69033B00E000237B61B8
:105C28004FF0FF32BB6902FA03F3DA43BB681A404C
:105C38007B699A404FF0FF317B6901FA03F3D9433E
:105C48007B680B40134318462437BD465DF8047B38
:105C58007047000080B582B000AF78607B68013B78
:105C6800B3F1807F01D301230FE00A4A7B68013B2F
:105C780053600F214FF0FF30FFF78EFF054B0022D6
:105C88009A60044B07221A60002318460837BD465D
:105C980080BD00BF10E000E080B582B000AF786042
:105CA8007868FFF729FF00BF0837BD4680BD80B57B
:105CB80086B000AF0346B9607A60FB7300237B614E
:105CC800FFF73EFF78617A68B9687869FFF78EFF59
:105CD800024697F90F3011461846FFF75DFF00BFDF
:105CE8001837BD4680BD80B582B000AF0346FB7152
:105CF80097F907301846FFF731FF00BF0837BD4650
:105D080080BD80B582B000AF78607868FFF7A2FFE9
:105D1800034618460837BD4680BD000080B487B0EA
:105D280000AF7860396000237B6154E13B681A68F2
:105D380001217B6901FA03F31340FB60FB68002B28
:105D480000F046813B685B6803F00303012B05D034
:105D58003B685B6803F00303022B30D17B689B68C8
:105D68003B617B695B00032202FA03F3DB433A6978
:105D780013403B613B68DA687B695B0002FA03F316
:105D88003A6913433B617B683A699A607B685B6850
:105D98003B6101227B6902FA03F3DB433A69134052
:105DA8003B613B685B681B0903F001027B6902FAEF
:105DB80003F33A6913433B617B683A695A603B686D
:105DC8005B6803F00303032B17D07B68DB683B6138
:105DD8007B695B00032202FA03F3DB433A69134051
:105DE8003B613B689A687B695B0002FA03F33A6996
:105DF80013433B617B683A69DA603B685B6803F090
:105E08000303022B23D17B69DA087B68083253F835
:105E180022303B617B6903F007039B000F2202FAE3
:105E280003F3DB433A6913403B613B681A697B69BA
:105E380003F007039B0002FA03F33A6913433B613B
:105E48007B69DA087B680832396943F822107B6875
:105E58001B683B617B695B00032202FA03F3DB43A7
:105E68003A6913403B613B685B6803F003027B6956
:105E78005B0002FA03F33A6913433B617B683A69B2
:105E88001A603B685B6803F44033002B00F0A08085
:105E9800584B9B69574A43F001039361554B9B69E3
:105EA80003F00103BB60BB68534A7B699B0802335C
:105EB80052F823303B617B6903F003039B000F22F8
:105EC80002FA03F3DB433A6913403B617B68B3F1A1
:105ED800904F19D07B68494A934213D07B68484A4F
:105EE80093420DD07B68474A934207D07B68464A65
:105EF800934201D1042308E0052306E0032304E0CC
:105F0800022302E0012300E000237A6902F0030281
:105F1800920093403A6913433B6137497B699B0878
:105F280002333A6941F82320384B9B683B61FB6890
:105F3800DB433A6913403B613B685B6803F48013B9
:105F4800002B03D03A69FB6813433B612F4A3B6936
:105F580093602E4BDB683B61FB68DB433A69134077
:105F68003B613B685B6803F40013002B03D03A697C
:105F7800FB6813433B61254A3B69D360234B5B684D
:105F88003B61FB68DB433A6913403B613B685B68F4
:105F980003F40033002B03D03A69FB6813433B61D9
:105FA8001A4A3B695360194B1B683B61FB68DB432A
:105FB8003A6913403B613B685B6803F48033002B0C
:105FC80003D03A69FB6813433B61104A3B6913608D
:105FD8007B6901337B613B681A687B6922FA03F3AA
:105FE800002B7FF4A3AE00BF00BF1C37BD465DF891
:105FF800047B704700100240000001400004004884
:1060080000080048000C0048001000480004014047
:1060180080B483B000AF78600B467B8013467B70FA
:106028007B78002B03D07A887B689A6102E07A88B3
:106038007B689A6200BF0C37BD465DF8047B7047E9
:1060480080B582B000AF78607B68002B01D1012356
:1060580081E07B6893F84130DBB2002B06D17B6886
:10606800002283F840207868FEF742FC7B682422EF
:1060780083F841207B681B681A687B681B6822F0DC
:1060880001021A607B685A687B681B6822F070629C
:106098001A617B681B689A687B681B6822F4004257
:1060A8009A607B68DB68012B07D17B689A687B68FC
:1060B8001B6842F400429A6006E07B689A687B6835
:1060C8001B6842F404429A607B68DB68022B04D1A7
:1060D8007B681B684FF400625A607B681B685B68CA
:1060E8007A68126843F0007343F4004353607B6896
:1060F8001B68DA687B681B6822F40042DA607B68F8
:106108001A697B685B6942EA03017B689B691A022A
:106118007B681B680A43DA607B68D9697B681A6AFE
:106128007B681B680A431A607B681B681A687B686F
:106138001B6842F001021A607B6800225A647B687F
:10614800202283F841207B6800221A637B680022A2
:1061580083F84220002318460837BD4680BD00005A
:1061680080B588B002AFF8607A601A460B467B812A
:1061780013463B81FB6893F84130DBB2202B40F09B
:10618800DA80FB6893F84030012B01D10223D3E079
:10619800FB68012283F84020FEF72EFE78617B69B8
:1061A8000093192301224FF40041F86800F0E6F942
:1061B8000346002B01D00123BEE0FB68212283F8AF
:1061C8004120FB68102283F84220FB6800225A64B1
:1061D800FB687A685A62FB683A895A85FB6800222C
:1061E8005A63FB685B8D9BB2FF2B0ED9FB68FF22BD
:1061F8001A85FB681B8DDAB27989514B00934FF0F1
:106208008073F86800F0F6FB6CE0FB685B8D9AB26F
:10621800FB681A85FB681B8DDAB27989484B0093B5
:106228004FF00073F86800F0E5FB5BE07A69396AC3
:10623800F86800F0F2F90346002B01D001237BE057
:10624800FB685B6A1A78FB681B689A62FB685B6A82
:106258005A1CFB685A62FB685B8D9BB2013B9AB281
:10626800FB685A85FB681B8D013B9AB2FB681A854F
:10627800FB685B8D9BB2002B34D0FB681B8D002B19
:1062880030D17B6900933B6A00228021F86800F0D6
:1062980075F90346002B01D001234DE0FB685B8DA7
:1062A8009BB2FF2B0ED9FB68FF221A85FB681B8D5A
:1062B800DAB27989002300934FF08073F86800F010
:1062C80099FB0FE0FB685B8D9AB2FB681A85FB6847
:1062D8001B8DDAB27989002300934FF00073F868B8
:1062E80000F088FBFB685B8D9BB2002B9ED17A691E
:1062F800396AF86800F0D8F90346002B01D0012369
:106308001AE0FB681B682022DA61FB681B68596881
:10631800FB681A680B4B0B405360FB68202283F81C
:106328004120FB68002283F84220FB68002283F8A2
:106338004020002300E0022318461837BD4680BDE0
:106348000020008000E800FE80B588B002AFF86049
:106358007A601A460B467B8113463B81FB6893F8AB
:106368004130DBB2202B40F0DB80FB6893F84030F3
:10637800012B01D10223D4E0FB68012283F84020DD
:10638800FEF73AFD78617B690093192301224FF4E7
:106398000041F86800F0F2F80346002B01D0012311
:1063A800BFE0FB68222283F84120FB68102283F8B3
:1063B8004220FB6800225A64FB687A685A62FB68CC
:1063C8003A895A85FB6800225A63FB685B8D9BB249
:1063D800FF2B0ED9FB68FF221A85FB681B8DDAB2EA
:1063E8007989524B00934FF08073F86800F002FBF4
:1063F8006DE0FB685B8D9AB2FB681A85FB681B8DA4
:10640800DAB27989494B00934FF00073F86800F0CD
:10641800F1FA5CE07A69396AF86800F089F90346AC
:10642800002B01D001237CE0FB681B685A6AFB68DB
:106438005B6AD2B21A70FB685B6A5A1CFB685A62C4
:10644800FB681B8D013B9AB2FB681A85FB685B8D64
:106458009BB2013B9AB2FB685A85FB685B8D9BB285
:10646800002B34D0FB681B8D002B30D17B69009347
:106478003B6A00228021F86800F080F80346002B70
:1064880001D001234DE0FB685B8D9BB2FF2B0ED939
:10649800FB68FF221A85FB681B8DDAB27989002315
:1064A80000934FF08073F86800F0A4FA0FE0FB68DF
:1064B8005B8D9AB2FB681A85FB681B8DDAB2798905
:1064C800002300934FF00073F86800F093FAFB681C
:1064D8005B8D9BB2002B9DD17A69396AF86800F010
:1064E800E3F80346002B01D001231AE0FB681B6880
:1064F8002022DA61FB681B685968FB681A680C4B34
:106508000B405360FB68202283F84120FB6800227F
:1065180083F84220FB68002283F84020002300E033
:10652800022318461837BD4680BD00BF00240080EE
:1065380000E800FE80B483B000AF78607B681B6819
:106548009B6903F00203022B03D17B681B680022BE
:106558009A627B681B689B6903F00103012B07D0D3
:106568007B681B689A697B681B6842F001029A6124
:1065780000BF0C37BD465DF8047B704780B584B01A
:1065880000AFF860B9603B601346FB7131E03B68CF
:10659800B3F1FF3F2DD0FEF72FFC0246BB69D31A9B
:1065A8003A689A4202D33B68002B22D1FB681B68E9
:1065B8009A69BB681340BA689A420CBF012300234A
:1065C800DBB21A46FB799A4213D1FB685B6C43F045
:1065D8002002FB685A64FB68202283F84120FB688C
:1065E800002283F84220FB68002283F84020012320
:1065F8000FE0FB681B689A69BB681340BA689A4247
:106608000CBF01230023DBB21A46FB799A42BED0A5
:10661800002318461037BD4680BD80B584B000AF52
:10662800F860B9607A6033E07A68B968F86800F0B1
:1066380001F90346002B01D0012331E0BB68B3F117
:10664800FF3F25D0FEF7D8FB02467B68D31ABA680D
:106658009A4202D3BB68002B1AD1FB681B689B695E
:1066680003F00203022B13D0FB685B6C43F020029B
:10667800FB685A64FB68202283F84120FB680022EB
:1066880083F84220FB68002283F84020012307E0BA
:10669800FB681B689B6903F00203022BC4D100232B
:1066A80018461037BD4680BD80B584B000AFF8608D
:1066B800B9607A602FE07A68B968F86800F0BAF8CB
:1066C8000346002B01D001232DE0FEF795FB02467F
:1066D8007B68D31ABA689A4202D3BB68002B1AD1D6
:1066E800FB681B689B6903F02003202B13D0FB6811
:1066F8005B6C43F02002FB685A64FB68202283F835
:106708004120FB68002283F84220FB68002283F8BE
:106718004020012307E0FB681B689B6903F0200306
:10672800202BC8D1002318461037BD4680BD000075
:1067380080B584B000AFF860B9607A606BE07A68C1
:10674800B968F86800F076F80346002B01D00123F9
:1067580069E0FB681B689B6903F02003202B38D194
:10676800FB681B689B6903F00403042B05D1FB68D5
:106778001B8D002B01D0002355E0FB681B689B692B
:1067880003F01003102B07D1FB681B681022DA6195
:10679800FB6804225A6402E0FB6800225A64FB6822
:1067A8001B682022DA61FB681B685968FB681A6855
:1067B8001F4B0B405360FB68202283F84120FB6885
:1067C800002283F84220FB68002283F8402001233E
:1067D80029E0FEF711FB02467B68D31ABA689A4291
:1067E80002D3BB68002B16D1FB681B689B6903F0BA
:1067F8000403042B0FD0FB685B6C43F02002FB689A
:106808005A64FB68202283F84120FB68002283F841
:106818004020012307E0FB681B689B6903F0040321
:10682800042B8CD1002318461037BD4680BD00BF0D
:1068380000E800FE80B58AB000AFF860B9607A6001
:10684800002387F82730FB681B689B69BB6100231E
:106858003B627B68FB61BB6903F01003002B68D0C7
:10686800FB681B681022DA6149E0BB68B3F1FF3F9F
:1068780045D0FEF7C1FA0246FB69D31ABA689A42B4
:1068880002D3BB68002B3AD1FB681B685B6803F432
:1068980080437B61FB6893F84230FB74FB681B689C
:1068A8009B6903F40043B3F5004F21D17B69B3F52D
:1068B800804F1DD0FB7C202B1AD0FB681B685A68C0
:1068C800FB681B6842F480425A60FEF795FAF8614B
:1068D8000EE0FEF791FA0246FB69D31A192B07D985
:1068E8003B6A43F020033B62012387F8273006E028
:1068F800FB681B689B6903F02003202BE9D1FB6828
:106908001B689B6903F02003202B03D097F82730DE
:10691800002BAAD097F82730002B03D1FB681B68FF
:106928002022DA613B6A43F004033B62012387F8C3
:106938002730FB681B689B69BB61BB6903F48073E4
:10694800002B0BD03B6A43F001033B62FB681B68DA
:106958004FF48072DA61012387F82730BB6903F4AA
:106968008063002B0BD03B6A43F008033B62FB6853
:106978001B684FF48062DA61012387F82730BB690E
:1069880003F40073002B0BD03B6A43F002033B6215
:10699800FB681B684FF40072DA61012387F827301F
:1069A80097F82730002B1CD0F868FFF7C3FDFB6869
:1069B8001B685968FB681A680D4B0B405360FB68ED
:1069C8005A6C3B6A1A43FB685A64FB68202283F8B6
:1069D8004120FB68002283F84220FB68002283F8EC
:1069E800402097F8273018462837BD4680BD00BF9D
:1069F80000E800FE80B487B000AFF8607B600B460B
:106A08007B8113467B727B89C3F309027B7A1B0463
:106A180003F47F031A437B681A433B6A134323F04A
:106A280000437B61FB681B685A683B6A5B0D03F493
:106A38008061084B0B43DB4302EA0301FB681B68D8
:106A48007A690A435A6000BF1C37BD465DF8047B6B
:106A5800704700BFFF63FF0380B483B000AF786066
:106A680039607B6893F84130DBB2202B38D17B68E2
:106A780093F84030012B01D1022332E07B680122D8
:106A880083F840207B68242283F841207B681B68B8
:106A98001A687B681B6822F001021A607B681B6811
:106AA8001A687B681B6822F480521A607B681B682E
:106AB80019687B681B683A680A431A607B681B6818
:106AC8001A687B681B6842F001021A607B68202202
:106AD80083F841207B68002283F84020002300E0EF
:106AE800022318460C37BD465DF8047B704780B416
:106AF80085B000AF786039607B6893F84130DBB2CD
:106B0800202B39D17B6893F84030012B01D1022327
:106B180033E07B68012283F840207B68242283F8D5
:106B280041207B681B681A687B681B6822F0010299
:106B38001A607B681B681B68FB60FB6823F4706342
:106B4800FB603B681B02FA681343FB607B681B68A9
:106B5800FA681A607B681B681A687B681B6842F0D1
:106B680001021A607B68202283F841207B6800229A
:106B780083F84020002300E0022318461437BD465E
:106B88005DF8047B7047000080B5ADF5007D00AF6F
:106B980007F50073A3F5FE73186007F50073A3F5F6
:106BA800FE731B68002B02D1012300F0F4BF07F528
:106BB8000073A3F5FE731B681B6803F00103002B29
:106BC80000F06D81B44B5B6803F00C03042B0CD010
:106BD800B14B5B6803F00C03082B57D1AE4B5B68D5
:106BE80003F48033B3F5803F50D14FF40033C7F836
:106BF800F031D7F8F03193FAA3F3C7F8EC31D7F8AE
:106C0800EC31B3FA83F3DBB23F2B02D8A24B1B68FB
:106C180015E04FF40033C7F8E831D7F8E83193FAB4
:106C2800A3F3C7F8E4314FF40033C7F8E031D7F8DD
:106C3800E03193FAA3F3C7F8DC31974B5B6A4FF462
:106C48000032C7F8D821D7F8D82192FAA2F2C7F8AB
:106C5800D421D7F8D421B2FA82F2D2B242F020027B
:106C6800D2B202F01F02012101FA02F21340002BF6
:106C780000F0148107F50073A3F5FE731B685B68C9
:106C8800002B40F00B81012300F085BF07F500734E
:106C9800A3F5FE731B685B68B3F5803F06D17E4B96
:106CA8001B687D4A43F48033136036E007F50073B0
:106CB800A3F5FE731B685B68002B0CD1764B1B6831
:106CC800754A23F480331360734B1B68724A23F4AC
:106CD8008023136021E007F50073A3F5FE731B689A
:106CE8005B68B3F5A02F0CD16B4B1B686A4A43F461
:106CF80080231360684B1B68674A43F48033136032
:106D08000BE0654B1B68644A23F480331360624BC5
:106D18001B68614A23F4802313605F4BDB6A23F00E
:106D28000F0207F50073A3F5FE731B689B685A49A9
:106D38001343CB6207F50073A3F5FE731B685B680A
:106D4800002B54D0FEF758F8C7F8F8010AE0FEF710
:106D580053F80246D7F8F831D31A642B02D9032323
:106D680000F019BF4FF40033C7F8D031D7F8D0314D
:106D780093FAA3F3C7F8CC31D7F8CC31B3FA83F33D
:106D8800DBB23F2B02D8444B1B6815E04FF40033AD
:106D9800C7F8C831D7F8C83193FAA3F3C7F8C43194
:106DA8004FF40033C7F8C031D7F8C03193FAA3F3D2
:106DB800C7F8BC31384B5B6A4FF40032C7F8B821CA
:106DC800D7F8B82192FAA2F2C7F8B421D7F8B421BB
:106DD800B2FA82F2D2B242F02002D2B202F01F021C
:106DE800012101FA02F21340002BB0D057E0FEF760
:106DF80003F8C7F8F8010AE0FDF7FEFF0246D7F8E6
:106E0800F831D31A642B02D9032300F0C4BE4FF41F
:106E18000033C7F8B031D7F8B03193FAA3F3C7F805
:106E2800AC31D7F8AC31B3FA83F3DBB23F2B02D8DD
:106E3800194B1B6815E04FF40033C7F8A831D7F891
:106E4800A83193FAA3F3C7F8A4314FF40033C7F875
:106E5800A031D7F8A03193FAA3F3C7F89C310E4BB1
:106E68005B6A4FF40032C7F89821D7F8982192FA54
:106E7800A2F2C7F89421D7F89421B2FA82F2D2B2DA
:106E880042F02002D2B202F01F02012101FA02F2FE
:106E98001340002BB0D102E00010024000BF07F5FC
:106EA8000073A3F5FE731B681B6803F00203002B35
:106EB80000F06C81CC4B5B6803F00C03002B0BD00B
:106EC800C94B5B6803F00C03082B6DD1C64B5B689C
:106ED80003F48033002B67D10223C7F89031D7F829
:106EE800903193FAA3F3C7F88C31D7F88C31B3FA01
:106EF80083F3DBB23F2B02D8BB4B1B6813E00223A2
:106F0800C7F88831D7F8883193FAA3F3C7F88431E2
:106F18000223C7F88031D7F8803193FAA3F3C7F872
:106F28007C31B14B5B6A0222C7F87821D7F8782107
:106F380092FAA2F2C7F87421D7F87421B2FA82F251
:106F4800D2B242F02002D2B202F01F02012101FAAD
:106F580002F21340002B0AD007F50073A3F5FE7365
:106F68001B681B69012B02D0012300F014BE9E4B45
:106F78001B6823F0F80207F50073A3F5FE731B687E
:106F88005B69F821C7F87011D7F8701191FAA1F16F
:106F9800C7F86C11D7F86C11B1FA81F1C9B28B40FE
:106FA800914913430B60F1E007F50073A3F5FE73F5
:106FB8001B681B69002B00F083800123C7F8683128
:106FC800D7F8683193FAA3F3C7F86431D7F8643176
:106FD800B3FA83F3DBB203F1845303F584139B0004
:106FE8001A4601231360FDF707FFC7F8F8010AE006
:106FF800FDF702FF0246D7F8F831D31A022B02D95F
:10700800032300F0C8BD0223C7F86031D7F8603108
:1070180093FAA3F3C7F85C31D7F85C31B3FA83F37A
:10702800DBB23F2B02D8704B1B6813E00223C7F872
:107038005831D7F8583193FAA3F3C7F854310223DB
:10704800C7F85031D7F8503193FAA3F3C7F84C3149
:10705800654B5B6A0222C7F84821D7F8482192FAA3
:10706800A2F2C7F84421D7F84421B2FA82F2D2B288
:1070780042F02002D2B202F01F02012101FA02F20C
:107088001340002BB4D0584B1B6823F0F80207F5C7
:107098000073A3F5FE731B685B69F821C7F84011FC
:1070A800D7F8401191FAA1F1C7F83C11D7F83C1173
:1070B800B1FA81F1C9B28B404B4913430B6065E0CB
:1070C8000123C7F83831D7F8383193FAA3F3C7F852
:1070D8003431D7F83431B3FA83F3DBB203F1845394
:1070E80003F584139B001A4600231360FDF784FE02
:1070F800C7F8F8010AE0FDF77FFE0246D7F8F83135
:10710800D31A022B02D9032300F045BD0223C7F886
:107118003031D7F8303193FAA3F3C7F82C31D7F8C8
:107128002C31B3FA83F3DBB23F2B02D82E4B1B680A
:1071380013E00223C7F82831D7F8283193FAA3F3CC
:10714800C7F824310223C7F82031D7F8203193FA41
:10715800A3F3C7F81C31244B5B6A0222C7F8182135
:10716800D7F8182192FAA2F2C7F81421D7F81421F7
:10717800B2FA82F2D2B242F02002D2B202F01F0278
:10718800012101FA02F21340002BB4D107F5007374
:10719800A3F5FE731B681B6803F00803002B00F0BF
:1071A800158107F50073A3F5FE731B689B69002B17
:1071B8007ED00123C7F81031D7F8103193FAA3F322
:1071C800C7F80C31D7F80C31B3FA83F3DBB21A469F
:1071D800064B13449B001A4601231360FDF70CFE6F
:1071E800C7F8F8010FE000BF00100240208190109E
:1071F800FDF702FE0246D7F8F831D31A022B02D95E
:10720800032300F0C8BC0223C7F80831D7F80831B7
:1072180093FAA3F3C7F8043107F50073A3F5807355
:1072280002221A6007F50073A3F580731B6893FAAE
:10723800A3F207F50073A3F582731A6007F50073CC
:10724800A3F5847302221A6007F50073A3F584730B
:107258001B6893FAA3F207F50073A3F586731A6007
:10726800B04B5A6A07F50073A3F5887302211960B9
:1072780007F50073A3F588731B6893FAA3F107F564
:107288000073A3F58A73196007F50073A3F58A7371
:107298001B68B3FA83F3DBB243F06003DBB203F09D
:1072A8001F03012101FA03F31340002BA0D08DE046
:1072B80007F50073A3F58C7301221A6007F50073B4
:1072C800A3F58C731B6893FAA3F207F50073A3F573
:1072D8008E731A6007F50073A3F58E731B68B3FAF3
:1072E80083F3DBB21A46904B13449B001A460023E3
:1072F8001360FDF781FDC7F8F8010AE0FDF77CFD92
:107308000246D7F8F831D31A022B02D9032300F02A
:1073180042BC07F50073A3F5907302221A6007F5C3
:107328000073A3F590731B6893FAA3F207F5007333
:10733800A3F592731A6007F50073A3F594730222FC
:107348001A6007F50073A3F594731B6893FAA3F208
:1073580007F50073A3F596731A6007F50073A3F594
:10736800987302221A6007F50073A3F598731B68D7
:1073780093FAA3F207F50073A3F59A731A60694BA1
:107388005A6A07F50073A3F59C730221196007F583
:107398000073A3F59C731B6893FAA3F107F50073B8
:1073A800A3F59E73196007F50073A3F59E731B6818
:1073B800B3FA83F3DBB243F06003DBB203F01F03DD
:1073C800012101FA03F31340002B97D107F500734D
:1073D800A3F5FE731B681B6803F00403002B00F081
:1073E8009E81002387F8FF314E4BDB6903F0805301
:1073F800002B16D14B4BDB694A4A43F08053D361CB
:10740800484BDB6903F0805207F50073A3F5FC7362
:107418001A6007F50073A3F5FC731B68012387F84E
:10742800FF31424B1B6803F48073002B1AD13F4B8A
:107438001B683E4A43F480731360FDF7DDFCC7F810
:10744800F80109E0FDF7D8FC0246D7F8F831D31A5D
:10745800642B01D903239EE3344B1B6803F4807328
:10746800002BEFD007F50073A3F5FE731B68DB68EC
:10747800012B06D12B4B1B6A2A4A43F001031362E6
:1074880035E007F50073A3F5FE731B68DB68002B76
:107498000CD1244B1B6A234A23F001031362214BAE
:1074A8001B6A204A23F00403136220E007F50073E7
:1074B800A3F5FE731B68DB68052B0CD1194B1B6AFF
:1074C800184A43F004031362164B1B6A154A43F02B
:1074D800010313620BE0134B1B6A124A23F00103EA
:1074E8001362104B1B6A0F4A23F00403136207F55B
:1074F8000073A3F5FE731B68DB68002B00F0878020
:10750800FDF77AFCC7F8F80112E0FDF775FC0246B2
:10751800D7F8F831D31A41F28832934208D90323B5
:1075280039E300BF00100240208190100070004035
:1075380007F50073A3F5A07302221A6007F500731C
:10754800A3F5A0731B6893FAA3F207F50073A3F5DC
:10755800A2731A6007F50073A3F5A47302221A60D8
:1075680007F50073A3F5A4731B6893FAA3F207F554
:107578000073A3F5A6731A6007F50073A3F5A67345
:107588001B68B3FA83F3DBB223F05F03DBB2002B93
:1075980002D1984B1B6A13E007F50073A3F5A87393
:1075A80002221A6007F50073A3F5A8731B6893FA03
:1075B800A3F207F50073A3F5AA731A608D4B5B6AF3
:1075C80007F50072A2F5AC720221116007F500728E
:1075D800A2F5AC72126892FAA2F107F50072A2F550
:1075E800AE72116007F50072A2F5AE721268B2FAB7
:1075F80082F2D2B242F04002D2B202F01F0201215E
:1076080001FA02F21340002B3FF47FAF7DE0FDF753
:10761800F3FBC7F8F8010BE0FDF7EEFB0246D7F8DD
:10762800F831D31A41F28832934201D90323B2E2E6
:1076380007F50073A3F5B07302221A6007F500730B
:10764800A3F5B0731B6893FAA3F207F50073A3F5CB
:10765800B2731A6007F50073A3F5B47302221A60B7
:1076680007F50073A3F5B4731B6893FAA3F207F543
:107678000073A3F5B6731A6007F50073A3F5B67324
:107688001B68B3FA83F3DBB223F05F03DBB2002B92
:1076980002D1584B1B6A13E007F50073A3F5B873C2
:1076A80002221A6007F50073A3F5B8731B6893FAF2
:1076B800A3F207F50073A3F5BA731A604D4B5B6A22
:1076C80007F50072A2F5BC720221116007F500727D
:1076D800A2F5BC72126892FAA2F107F50072A2F53F
:1076E800BE72116007F50072A2F5BE721268B2FA96
:1076F80082F2D2B242F04002D2B202F01F0201215D
:1077080001FA02F21340002B86D197F8FF31012BC2
:1077180005D1384BDB69374A23F08053D36107F52D
:107728000073A3F5FE731B68DB69002B00F032823F
:10773800304B5B6803F00C03082B00F0018207F55F
:107748000073A3F5FE731B68DB69022B40F05781B9
:1077580007F50073A3F5C0734FF080721A6007F540
:107768000073A3F5C0731B6893FAA3F207F50073BF
:10777800A3F5C2731A6007F50073A3F5C2731B68FB
:10778800B3FA83F3DBB203F1845303F584139B004C
:107798001A4600231360FDF72FFBC7F8F80109E02C
:1077A800FDF72AFB0246D7F8F831D31A022B01D984
:1077B8000323F0E107F50073A3F5C4734FF00072DB
:1077C8001A6007F50073A3F5C4731B6893FAA3F254
:1077D80007F50073A3F5C6731A6007F50073A3F5E0
:1077E800C6731B68B3FA83F3DBB23F2B04D8014B93
:1077F8001B6829E00010024007F50073A3F5C87361
:107808004FF000721A6007F50073A3F5C8731B6880
:1078180093FAA3F207F50073A3F5CA731A6007F584
:107828000073A3F5CC734FF000721A6007F500736C
:10783800A3F5CC731B6893FAA3F207F50073A3F5BD
:10784800CE731A60C34B5B6A07F50072A2F5D0725B
:107858004FF00071116007F50072A2F5D07212683E
:1078680092FAA2F107F50072A2F5D272116007F53B
:107878000072A2F5D2721268B2FA82F2D2B242F063
:107888002002D2B202F01F02012101FA02F21340D3
:10789800002B85D1AF4B5B6823F4741207F5007396
:1078A800A3F5FE731B68596A07F50073A3F5FE7309
:1078B8001B681B6A0B43A74913434B6007F500730A
:1078C800A3F5D4734FF080721A6007F50073A3F51F
:1078D800D4731B6893FAA3F207F50073A3F5D67364
:1078E8001A6007F50073A3F5D6731B68B3FA83F320
:1078F800DBB203F1845303F584139B001A4601237A
:107908001360FDF779FAC7F8F80109E0FDF774FA92
:107918000246D7F8F831D31A022B01D903233AE1EA
:1079280007F50073A3F5D8734FF000721A6007F5D6
:107938000073A3F5D8731B6893FAA3F207F50073D5
:10794800A3F5DA731A6007F50073A3F5DA731B68F9
:10795800B3FA83F3DBB23F2B02D87E4B1B6827E0D8
:1079680007F50073A3F5DC734FF000721A6007F592
:107978000073A3F5DC731B6893FAA3F207F5007391
:10798800A3F5DE731A6007F50073A3F5E0734FF0F3
:1079980000721A6007F50073A3F5E0731B6893FA89
:1079A800A3F207F50073A3F5E2731A60694B5B6AEB
:1079B80007F50072A2F5E4724FF00071116007F547
:1079C8000072A2F5E472126892FAA2F107F5007249
:1079D800A2F5E672116007F50072A2F5E672126868
:1079E800B2FA82F2D2B242F02002D2B202F01F0200
:1079F800012101FA02F21340002B87D0CAE007F5F3
:107A08000073A3F5E8734FF080721A6007F50073EE
:107A1800A3F5E8731B6893FAA3F207F50073A3F5BF
:107A2800EA731A6007F50073A3F5EA731B68B3FAE3
:107A380083F3DBB203F1845303F584139B001A46E6
:107A480000231360FDF7D8F9C7F8F80109E0FDF73E
:107A5800D3F90246D7F8F831D31A022B01D90323F8
:107A680099E007F50073A3F5EC734FF000721A6004
:107A780007F50073A3F5EC731B6893FAA3F207F5F7
:107A88000073A3F5EE731A6007F50073A3F5EE73A0
:107A98001B68B3FA83F3DBB23F2B02D82D4B1B686C
:107AA80027E007F50073A3F5F0734FF000721A6032
:107AB80007F50073A3F5F0731B6893FAA3F207F5B3
:107AC8000073A3F5F2731A6007F50073A3F5F47356
:107AD8004FF000721A6007F50073A3F5F4731B6882
:107AE80093FAA3F207F50073A3F5F6731A60194B1E
:107AF8005B6A07F50072A2F5F8724FF00071116029
:107B080007F50072A2F5F872126892FAA2F107F569
:107B18000072A2F5FA72116007F50072A2F5FA7206
:107B28001268B2FA82F2D2B242F02002D2B202F065
:107B38001F02012101FA02F21340002B87D129E02C
:107B480007F50073A3F5FE731B68DB69012B03D1EE
:107B5800012320E000100240114B5B68C7F8F431A4
:107B6800D7F8F43103F4803207F50073A3F5FE73F8
:107B78001B681B6A9A420BD1D7F8F43103F47012D0
:107B880007F50073A3F5FE731B685B6A9A4201D080
:107B9800012300E00023184607F50077BD4680BDA5
:107BA8000010024080B59EB000AF786039600023B5
:107BB8007B677B68002B01D1012354E1894B1B684B
:107BC80003F007033A689A4210D9864B1B6823F0E2
:107BD800070284493B6813430B60824B1B6803F020
:107BE80007033A689A4201D001233CE17B681B688D
:107BF80003F00203002B08D07B4B5B6823F0F002F4
:107C08007B689B68784913434B607B681B6803F06B
:107C18000103002B00F0CD807B685B68012B37D116
:107C28004FF40033FB66FB6E93FAA3F33B673B6F9D
:107C3800B3FA83F3DBB23F2B02D86B4B1B680FE020
:107C48004FF40033BB66BB6E93FAA3F37B664FF425
:107C580000333B663B6E93FAA3F3FB65624B5B6AAA
:107C68004FF40032BA65BA6D92FAA2F27A657A6D6B
:107C7800B2FA82F2D2B242F02002D2B202F01F026D
:107C8800012101FA02F21340002B71D10123EAE02D
:107C98007B685B68022B37D14FF000733B653B6D07
:107CA80093FAA3F3FB64FB6CB3FA83F3DBB23F2BC9
:107CB80002D84D4B1B680FE04FF00073BB64BB6CE0
:107CC80093FAA3F37B644FF000733B643B6C93FA25
:107CD800A3F3FB63444B5B6A4FF00072BA63BA6B61
:107CE80092FAA2F27A637A6BB2FA82F2D2B242F0D4
:107CF8002002D2B202F01F02012101FA02F213405F
:107D0800002B35D10123AEE002233B633B6B93FA92
:107D1800A3F3FB62FB6AB3FA83F3DBB23F2B02D80F
:107D2800314B1B680DE00223BB62BB6A93FAA3F3D5
:107D38007B6202233B623B6A93FAA3F3FB612A4B03
:107D48005B6A0222BA61BA6992FAA2F27A617A6926
:107D5800B2FA82F2D2B242F02002D2B202F01F028C
:107D6800012101FA02F21340002B01D101237AE02C
:107D78001D4B5B6823F003027B685B681A49134359
:107D88004B60FDF739F878670AE0FDF735F80246E9
:107D98007B6FD31A41F28832934201D9032362E000
:107DA800114B5B6803F00C027B685B689B009A428E
:107DB800EBD10C4B1B6803F007033A689A4215D2C3
:107DC800084B1B6823F0070206493B6813430B6006
:107DD800044B1B6803F007033A689A4206D0012354
:107DE80041E000BF00200240001002407B681B6891
:107DF80003F00403002B08D01D4B5B6823F4E062FA
:107E08007B68DB681A4913434B607B681B6803F087
:107E18000803002B09D0164B5B6823F460527B687B
:107E28001B69DB00124913434B6000F029F8014637
:107E38000F4B5B6803F0F003F0223A613A6992FA5B
:107E4800A2F2FA60FA68B2FA82F2D2B2D340094AD0
:107E5800D35C21FA03F3084A1360084B1B681846E1
:107E6800FCF786FF002318467837BD4680BD00BF63
:107E780000100240309900085C00002060000020DB
:107E880080B48BB000AF0023FB610023BB610023EB
:107E98007B6200237B6100233B62294B5B68FB61AB
:107EA800FB6903F00C03042B02D0082B03D03CE041
:107EB800244B3B623CE0FB6903F470134FF47012EF
:107EC800BA60BA6892FAA2F27A607A68B2FA82F272
:107ED800D2B2D3401C4AD35C7B61194BDB6A03F0F6
:107EE8000F030F223A613A6992FAA2F2FA60FA682D
:107EF800B2FA82F2D2B2D340144AD35CBB61FB69B6
:107F080003F48033002B08D00E4ABB69B2FBF3F2AE
:107F18007B6902FB03F37B6204E07B690C4A02FB8A
:107F280003F37B627B6A3B6202E00A4B3B6200BF61
:107F38003B6A18462C37BD465DF8047B704700BF86
:107F4800001002400024F4004099000850990008ED
:107F580000093D0000127A0080B592B000AF786049
:107F680000233B640023FB63002387F847307B68CA
:107F78001B6803F48033002B00F0D2804D4BDB6983
:107F880003F08053002B0ED14A4BDB69494A43F07A
:107F98008053D361474BDB6903F08053BB60BB68F8
:107FA800012387F84730444B1B6803F48073002B88
:107FB80018D1414B1B68404A43F480731360FCF7A7
:107FC8001BFF386408E0FCF717FF02463B6CD31A26
:107FD800642B01D9032349E1374B1B6803F48073F1
:107FE800002BF0D0334B1B6A03F44073FB63FB6B2D
:107FF800002B00F082807B685B6803F44073FA6BA7
:108008009A427AD02B4B1B6A23F44073FB634FF4DC
:1080180080333B633B6B93FAA3F3FB62FB6AB3FACF
:1080280083F3DBB21A46254B13449B001A460123FF
:1080380013604FF48033BB63BB6B93FAA3F37B638A
:108048007B6BB3FA83F3DBB21A461C4B13449B00D9
:108058001A4600231360174AFB6B1362FB6B03F08D
:108068000103002B49D0FCF7C7FE38640AE0FCF78F
:10807800C3FE02463B6CD31A41F28832934201D9BF
:108088000323F3E00223BB62BB6A93FAA3F37B6288
:1080980002233B623B6A93FAA3F3FB61FB69B3FAE1
:1080A80083F3DBB223F05F03DBB2002B08D1014B73
:1080B8001B6A0DE000100240007000400081901023
:1080C8000223BB61BB6993FAA3F37B61694B5B6ACB
:1080D80002223A613A6992FAA2F2FA60FA68B2FAAE
:1080E80082F2D2B242F04002D2B202F01F02012163
:1080F80001FA02F21340002BB9D05E4B1B6A23F43D
:1081080040727B685B685B4913430B6297F84730A2
:10811800012B05D1574BDB69564A23F08053D361B5
:108128007B681B6803F00103002B08D0514B1B6BC5
:1081380023F003027B689B684E4913430B637B68FB
:108148001B6803F00203002B08D04A4B1B6B23F477
:1081580040327B68DB68474913430B637B681B68C5
:1081680003F00403002B08D0424B1B6B23F440227E
:108178007B681B693F4913430B637B681B6803F0EB
:108188002003002B08D03B4B1B6B23F010027B68AD
:10819800DB69384913430B637B681B6803F40033BE
:1081A800002B08D0334B5B6823F480027B681B6B81
:1081B800304913434B607B681B6803F04003002B76
:1081C80008D02C4B1B6B23F020027B681B6A2949C3
:1081D80013430B637B681B6803F00803002B08D06C
:1081E800244B1B6B23F440127B685B6921491343C2
:1081F8000B637B681B6803F01003002B08D01D4B32
:108208001B6B23F440027B689B691A4913430B6379
:108218007B681B6803F40073002B08D0154B5B6860
:1082280023F400027B689B6A124913434B607B6806
:108238001B6803F08003002B08D00E4BDB6A23F485
:10824800F8727B685B6A0B491343CB627B681B68D7
:1082580003F48053002B08D0064B1B6B23F4807269
:108268007B68DB6A034913430B63002318464837CE
:10827800BD4680BD0010024080B584B000AF786074
:108288007B68002B01D101239DE07B685B6A002B92
:1082980008D17B685B68B3F5827F09D07B680022D0
:1082A800DA6105E07B6800221A617B6800225A6166
:1082B8007B6800229A627B6893F85D30DBB2002B02
:1082C80006D17B68002283F85C207868FCF7A4FB61
:1082D8007B68022283F85D207B681B681A687B68CC
:1082E8001B6822F040021A607B68DB68B3F5E06F18
:1082F80002D90023FB6002E04FF48053FB607B68E7
:10830800DB68B3F5706F07D07B68DB68B3F5E06FA7
:1083180002D07B6800229A627B685B6803F48272F1
:108328007B689B6803F404431A437B681B6903F06A
:1083380002031A437B685B6903F001031A437B68F5
:108348009B6903F400731A437B68DB6903F0380305
:108358001A437B681B6A03F0800342EA03017B68C7
:108368009B6A03F400527B681B680A431A607B68A7
:108378009B691B0C03F004027B685B6A03F0100323
:108388001A437B685B6B03F008031A437B68DB685E
:1083980003F4706342EA0301FB6803F480527B68CC
:1083A8001B680A435A607B681B68DA697B681B682C
:1083B80022F40062DA617B6800221A667B68012277
:1083C80083F85D20002318461037BD4680BD80B570
:1083D8008AB000AFF860B9607A607B8001237B6265
:1083E800002387F82330FB6893F85C30012B01D118
:1083F80002230AE2FB68012283F85C20FCF7FCFCFC
:10840800F861FB6893F85D30FB76FB685B687B611D
:108418007B887B827B883B82FB7E012B0ED07B692D
:10842800B3F5827F06D1FB689B68002B02D1FB7EE7
:10843800042B03D0022387F82330E0E1BB68002B2C
:1084480005D07B68002B02D07B88002B03D1012349
:1084580087F82330D3E1FB6893F85D30DBB2042B57
:1084680003D0FB68052283F85D20FB6800221A66AA
:10847800FB687A681A64FB687A88A3F84620FB6868
:108488007A88A3F84420FB68BA689A63FB687A88FC
:10849800DA87FB687A889A87FB680022DA64FB68C7
:1084A80000221A65FB68DB68B3F5E06F02D83B8AE7
:1084B800012B08D9FB681B685A68FB681B6822F403
:1084C80080525A6007E0FB681B685A68FB681B68A3
:1084D80042F480525A60FB681B681B6803F0400333
:1084E800402B07D0FB681B681A68FB681B6842F0C2
:1084F80040021A60FB68DB68B3F5E06F40F28180E8
:10850800FB685B68002B02D07B8A012B6DD1FB686E
:108518009B6B1A88FB681B68DA60FB689B6B9A1C6C
:10852800FB689A63FB68DB8F9BB2013B9AB2FB68DE
:10853800DA875AE0FB681B689B6803F00203022B8A
:108548001BD1FB68DB8F9BB2002B16D07B6A012BFB
:1085580013D1FB689B6B1A88FB681B68DA60FB68A1
:108568009B6B9A1CFB689A63FB68DB8F9BB2013B91
:108578009AB2FB68DA8700237B62FB681B689B68FA
:1085880003F00103012B1CD1FB68B3F846309BB202
:10859800002B16D0FB681B68DA68FB681B6C92B26C
:1085A8001A80FB681B6C9A1CFB681A64FB68B3F89A
:1085B80046309BB2013B9AB2FB68A3F846200123E0
:1085C8007B62FCF719FC0246FB69D31A3A6B9A42A4
:1085D8000BD83B6BB3F1FF3F07D0032387F8233059
:1085E800FB68012283F85D2009E1FB68DB8F9BB201
:1085F800002B9FD1FB68B3F846309BB2002B99D172
:10860800E3E0FB685B68002B03D07B8A012B40F01A
:10861800CF80FB68DB8F9BB2012B12D9FB689B6B69
:108628001A88FB681B68DA60FB689B6B9A1CFB68FE
:108638009A63FB68DB8F9BB2023B9AB2FB68DA87CE
:10864800B6E0FB689A6BFB681B680C3312781A70EB
:10865800FB689B6B5A1CFB689A63FB68DB8F9BB2B9
:10866800013B9AB2FB68DA87A2E0FB681B689B684B
:1086780003F00203022B34D1FB68DB8F9BB2002B83
:108688002FD07B6A012B2CD1FB68DB8F9BB2012B8F
:1086980012D9FB689B6B1A88FB681B68DA60FB6859
:1086A8009B6B9A1CFB689A63FB68DB8F9BB2023B4F
:1086B8009AB2FB68DA8712E0FB689A6BFB681B6862
:1086C8000C3312781A70FB689B6B5A1CFB689A6310
:1086D800FB68DB8F9BB2013B9AB2FB68DA87002309
:1086E8007B62FB681B689B6803F00103012B48D180
:1086F800FB68B3F846309BB2002B42D0FB68B3F856
:1087080046309BB2012B23D9FB681B68DA68FB68EB
:108718001B6C92B21A80FB681B6C9A1CFB681A646B
:10872800FB68B3F846309BB2023B9AB2FB68A3F8E9
:108738004620FB68B3F846309BB2012B1FD8FB6874
:108748001B685A68FB681B6842F480525A6016E03E
:10875800FB681B6803F10C02FB681B6C1278D2B231
:108768001A70FB681B6C5A1CFB681A64FB68B3F828
:1087780046309BB2013B9AB2FB68A3F8462001231E
:108788007B62FCF739FB0246FB69D31A3A6B9A42C3
:1087980003D83B6BB3F1FF3F02D13B6B002B07D1F2
:1087A800032387F82330FB68012283F85D2026E045
:1087B800FB68DB8F9BB2002B7FF457AFFB68B3F8E5
:1087C80046309BB2002B7FF450AFFA69396BF868DA
:1087D80000F03EF90346002B05D0012387F823302B
:1087E800FB6820221A66FB681B6E002B03D001234E
:1087F80087F8233003E0FB68012283F85D20FB68DB
:10880800002283F85C2097F8233018462837BD46A5
:1088180080BD000080B588B000AFF860B9603B60EB
:108828001346FB71FCF7E8FA0246BB6A9B1A3A68E2
:108838001344FB61FCF7E0FAB861394B1B685B0134
:108848001B0DFA6902FB03F37B6154E03B68B3F14B
:10885800FF3F50D0FCF7D0FA0246BB69D31AFA6939
:108868009A4202D9FB69002B3DD1FB681B685A6804
:10887800FB681B6822F0E0025A60FB685B68B3F58E
:10888800827F11D1FB689B68B3F5004F04D0FB6869
:108898009B68B3F5806F07D1FB681B681A68FB6893
:1088A8001B6822F040021A60FB689B6AB3F5005F00
:1088B8000FD1FB681B681A68FB681B6822F400521A
:1088C8001A60FB681B681A68FB681B6842F4005250
:1088D8001A60FB68012283F85D20FB68002283F898
:1088E8005C20032317E07B69002B01D10023FB6187
:1088F8007B69013B7B61FB681B689A68BB68134016
:10890800BA689A420CBF01230023DBB21A46FB79EE
:108918009A429BD1002318462037BD4680BD00BF30
:108928005C00002080B58AB000AFF860B9607A605A
:108938003B600023FB75FCF75FFA02463B6B9B1A12
:108948003A6813447B62FCF757FA3862FB681B6885
:108958000C33FB613D4B1A6813469B001344DA0045
:10896800D31A1B0D7A6A02FB03F3BB6160E0BB6894
:10897800B3F5C06F07D17B68002B04D1FB691B7866
:10898800DBB2FB75FB7D3B68B3F1FF3F50D0FCF7D2
:1089980033FA02463B6AD31A7A6A9A4202D97B6A48
:1089A800002B3DD1FB681B685A68FB681B6822F0E6
:1089B800E0025A60FB685B68B3F5827F11D1FB68FF
:1089C8009B68B3F5004F04D0FB689B68B3F5806FD4
:1089D80007D1FB681B681A68FB681B6822F0400215
:1089E8001A60FB689B6AB3F5005F0FD1FB681B68D0
:1089F8001A68FB681B6822F400521A60FB681B683F
:108A08001A68FB681B6842F400521A60FB6801226E
:108A180083F85D20FB68002283F85C20032310E0C4
:108A2800BB69002B01D100237B62BB69013BBB61A1
:108A3800FB681B689A68BB6813407A689A4296D1AB
:108A4800002318462837BD4680BD00BF5C000020C3
:108A580080B586B002AFF860B9607A607B68009331
:108A6800BB6800224FF4C051F868FFF75BFF03466C
:108A7800002B07D0FB681B6E43F02002FB681A66C8
:108A8800032327E07B680093BB6800228021F868F5
:108A9800FFF7C0FE0346002B07D0FB681B6E43F0B0
:108AA8002002FB681A66032314E07B680093BB6806
:108AB80000224FF4C061F868FFF734FF0346002B2B
:108AC80007D0FB681B6E43F02002FB681A6603237D
:108AD80000E0002318461037BD4680BD80B582B03F
:108AE80000AF78607B68002B01D1012349E07B68E7
:108AF80093F83D30DBB2002B06D17B68002283F867
:108B08003C207868FBF7CAFF7B68022283F83D2087
:108B18007B681A687B6804331946104600F03EFAF1
:108B28007B68012283F848207B68012283F83E2075
:108B38007B68012283F83F207B68012283F840206C
:108B48007B68012283F841207B68012283F8422058
:108B58007B68012283F843207B68012283F8442044
:108B68007B68012283F845207B68012283F8462030
:108B78007B68012283F847207B68012283F83D2027
:108B8800002318460837BD4680BD000080B584B074
:108B980000AF786039603B68002B09D17B6893F897
:108BA8003E30DBB2012B14BF01230023DBB23CE0D3
:108BB8003B68042B09D17B6893F83F30DBB2012B6B
:108BC80014BF01230023DBB22FE03B68082B09D137
:108BD8007B6893F84030DBB2012B14BF01230023DC
:108BE800DBB222E03B680C2B09D17B6893F841305B
:108BF800DBB2012B14BF01230023DBB215E03B6875
:108C0800102B09D17B6893F84230DBB2012B14BFDB
:108C180001230023DBB208E07B6893F84330DBB222
:108C2800012B14BF01230023DBB2002B01D0012349
:108C38008DE03B68002B04D17B68022283F83E203C
:108C480023E03B68042B04D17B68022283F83F2091
:108C58001BE03B68082B04D17B68022283F8402084
:108C680013E03B680C2B04D17B68022283F8412077
:108C78000BE03B68102B04D17B68022283F842206A
:108C880003E07B68022283F843207B681B6801228B
:108C98003968184600F0AAFC7B681B682E4A934284
:108CA8000ED07B681B682D4A934209D07B681B68ED
:108CB8002B4A934204D07B681B682A4A934201D10D
:108CC800012300E00023002B07D07B681B685A6C47
:108CD8007B681B6842F400425A647B681B681E4A22
:108CE800934213D07B681B68B3F1804F0ED07B682A
:108CF8001B681D4A934209D07B681B681B4A934234
:108D080004D07B681B68154A934215D17B681B68A1
:108D18009A68174B1340FB60FB68062B15D0FB685D
:108D2800B3F5803F11D07B681B681A687B681B68A5
:108D380042F001021A6008E07B681B681A687B68C9
:108D48001B6842F001021A6000E000BF00231846C9
:108D58001037BD4680BD00BF002C014000400140D7
:108D68000044014000480140000400400008004061
:108D78000700010080B586B000AFF860B9607A607E
:108D88000023FB75FB6893F83C30012B01D10223CB
:108D9800FFE0FB68012283F83C207B68142B00F27B
:108DA800F08001A252F823F0058E00088B8F00088E
:108DB8008B8F00088B8F0008458E00088B8F00086A
:108DC8008B8F00088B8F0008878E00088B8F000818
:108DD8008B8F00088B8F0008C78E00088B8F0008C8
:108DE8008B8F00088B8F0008098F00088B8F000875
:108DF8008B8F00088B8F0008498F0008FB681B6861
:108E0800B968184600F04CF9FB681B689A69FB685A
:108E18001B6842F008029A61FB681B689A69FB6844
:108E28001B6822F004029A61FB681B689969BB6899
:108E38001A69FB681B680A439A61A5E0FB681B680E
:108E4800B968184600F0B2F9FB681B689A69FB68B4
:108E58001B6842F400629A61FB681B689A69FB68A8
:108E68001B6822F480629A61FB681B689969BB6879
:108E78001B691A02FB681B680A439A6184E0FB6855
:108E88001B68B968184600F011FAFB681B68DA69B4
:108E9800FB681B6842F00802DA61FB681B68DA6944
:108EA800FB681B6822F00402DA61FB681B68D96959
:108EB800BB681A69FB681B680A43DA6164E0FB68EF
:108EC8001B68B968184600F06FFAFB681B68DA6916
:108ED800FB681B6842F40062DA61FB681B68DA69A8
:108EE800FB681B6822F48062DA61FB681B68D96939
:108EF800BB681B691A02FB681B680A43DA6143E016
:108F0800FB681B68B968184600F0B2FAFB681B6872
:108F18005A6DFB681B6842F008025A65FB681B68BB
:108F28005A6DFB681B6822F004025A65FB681B68CF
:108F3800596DBB681A69FB681B680A435A6523E0C8
:108F4800FB681B68B968184600F0F0FAFB681B68F4
:108F58005A6DFB681B6842F400625A65FB681B681F
:108F68005A6DFB681B6822F480625A65FB681B68AF
:108F7800596DBB681B691A02FB681B680A435A656E
:108F880002E00123FB7500BFFB68002283F83C2048
:108F9800FB7D18461837BD4680BD00BF80B485B03C
:108FA80000AF786039607B681B68FB607B68364A75
:108FB80093420BD07B68B3F1804F07D07B68334A6C
:108FC800934203D07B68324A934208D1FB6823F06E
:108FD8007003FB603B685B68FA681343FB607B685F
:108FE800294A934217D07B68B3F1804F13D07B682E
:108FF800264A93420FD07B68254A93420BD07B6860
:10900800244A934207D07B68234A934203D07B6863
:10901800224A934208D1FB6823F44073FB603B6803
:10902800DB68FA681343FB60FB6823F080023B6847
:109038005B691343FB607B68FA681A603B689A684F
:109048007B68DA623B681A687B689A627B680E4ABA
:1090580093420BD07B680F4A934207D07B680E4A35
:10906800934203D07B680D4A934203D13B681A6947
:109078007B681A637B6801225A6100BF1437BD46BA
:109088005DF8047B704700BF002C014000040040DD
:1090980000080040004001400044014000480140F1
:1090A80080B487B000AF786039607B681B6A23F0B2
:1090B80001027B681A627B681B6A7B617B685B685C
:1090C8003B617B689B69FB60FB6823F4803323F07A
:1090D8007003FB60FB6823F00303FB603B681B68BD
:1090E800FA681343FB607B6923F002037B613B68EA
:1090F8009B687A6913437B617B68284A93420BD04B
:109108007B68274A934207D07B68264A934203D05C
:109118007B68254A93420CD17B6923F008037B6165
:109128003B68DB687A6913437B617B6923F004033E
:109138007B617B68194A93420BD07B68184A93423B
:1091480007D07B68174A934203D07B68164A93423C
:1091580011D13B6923F480733B613B6923F40073AD
:109168003B613B685B693A6913433B613B689B69B8
:109178003A6913433B617B683A695A607B68FA68CD
:109188009A613B685A687B685A637B687A691A6295
:1091980000BF1C37BD465DF8047B7047002C0140BA
:1091A80000400140004401400048014080B487B0BD
:1091B80000AF786039607B681B6A23F010027B6817
:1091C8001A627B681B6A7B617B685B683B617B68B2
:1091D8009B69FB60FB6823F0807323F4E043FB602A
:1091E800FB6823F44073FB603B681B681B02FA684A
:1091F8001343FB607B6923F020037B613B689B681A
:109208001B017A6913437B617B68244A93420DD121
:109218007B6923F080037B613B68DB681B017A690B
:1092280013437B617B6923F040037B617B681B4AA6
:1092380093420BD07B681A4A934207D07B68194A3D
:10924800934203D07B68184A934213D13B6923F4B5
:1092580080633B613B6923F400633B613B685B6966
:109268009B003A6913433B613B689B699B003A69E1
:1092780013433B617B683A695A607B68FA689A6174
:109288003B685A687B689A637B687A691A6200BF90
:109298001C37BD465DF8047B704700BF002C0140B9
:1092A80000400140004401400048014080B487B0BC
:1092B80000AF786039607B681B6A23F480727B6832
:1092C8001A627B681B6A7B617B685B683B617B68B1
:1092D800DB69FB60FB6823F4803323F07003FB60D9
:1092E800FB6823F00303FB603B681B68FA681343C1
:1092F800FB607B6923F400737B613B689B681B02FE
:109308007A6913437B617B68234A93420DD17B6959
:1093180023F400637B613B68DB681B027A691343B3
:109328007B617B6923F480637B617B681A4A934283
:109338000BD07B68194A934207D07B68184A93423E
:1093480003D07B68174A934213D13B6923F48053B7
:109358003B613B6923F400533B613B685B691B013C
:109368003A6913433B613B689B691B013A691343A4
:109378003B617B683A695A607B68FA68DA613B68E6
:109388005A687B68DA637B687A691A6200BF1C379F
:10939800BD465DF8047B7047002C01400040014049
:1093A800004401400048014080B487B000AF7860B5
:1093B80039607B681B6A23F480527B681A627B6879
:1093C8001B6A3B617B685B687B617B68DB69FB6070
:1093D800FB6823F0807323F4E043FB60FB6823F40D
:1093E8004073FB603B681B681B02FA681343FB6011
:1093F8003B6923F400533B613B689B681B033A6954
:1094080013433B617B68164A93420BD07B68154A2D
:10941800934207D07B68144A934203D07B68134A6F
:10942800934209D17B6923F480437B613B685B6984
:109438009B017A6913437B617B687A695A607B6810
:10944800FA68DA613B685A687B681A647B683A692B
:109458001A6200BF1C37BD465DF8047B704700BF29
:10946800002C0140004001400044014000480140F8
:1094780080B487B000AF786039607B681B6A23F4DA
:1094880080327B681A627B681B6A3B617B685B6819
:109498007B617B685B6DFB60FB6823F4803323F0A2
:1094A8007003FB603B681B68FA681343FB603B6909
:1094B80023F400333B613B689B681B043A69134300
:1094C8003B617B68154A93420BD07B68144A9342F0
:1094D80007D07B68134A934203D07B68124A9342B1
:1094E80009D17B6923F480337B613B685B691B028C
:1094F8007A6913437B617B687A695A607B68FA688A
:109508005A653B685A687B689A657B683A691A624B
:1095180000BF1C37BD465DF8047B7047002C014036
:1095280000400140004401400048014080B487B039
:1095380000AF786039607B681B6A23F480127B680F
:109548001A627B681B6A3B617B685B687B617B682E
:109558005B6DFB60FB6823F0807323F4E043FB60E2
:109568003B681B681B02FA681343FB603B6923F4E2
:1095780000133B613B689B681B053A6913433B61D9
:109588007B68164A93420BD07B68154A934207D0F2
:109598007B68144A934203D07B68134A934209D1EB
:1095A8007B6923F480237B613B685B699B027A6952
:1095B80013437B617B687A695A607B68FA685A65ED
:1095C8003B685A687B68DA657B683A691A6200BF4B
:1095D8001C37BD465DF8047B704700BF002C014076
:1095E80000400140004401400048014080B487B079
:1095F80000AFF860B9607A60BB6803F01F0301220E
:1096080002FA03F37B61FB681A6A7B69DB431A4041
:10961800FB681A62FB681A6ABB6803F01F03796863
:1096280001FA03F31A43FB681A6200BF1C37BD46F0
:109638005DF8047B7047000080B485B000AF7860A7
:1096480039607B6893F83C30012B01D1022359E043
:109658007B68012283F83C207B68022283F83D2046
:109668007B681B685B68FB607B681B689B68BB60EA
:109678007B681B68264A934208D1FB6823F4700371
:10968800FB603B685B68FA681343FB60FB6823F088
:109698007003FB603B681B68FA681343FB607B68D8
:1096A8001B68FA685A607B681B68194A934213D092
:1096B8007B681B68B3F1804F0ED07B681B68154A26
:1096C800934209D07B681B68134A934204D07B6895
:1096D8001B68124A93420CD1BB6823F08003BB601D
:1096E8003B689B68BA681343BB607B681B68BA68B1
:1096F8009A607B68012283F83D207B68002283F80A
:109708003C20002318461437BD465DF8047B70479B
:10971800002C0140000400400008004000400140C7
:1097280080B485B000AF786039600023FB607B6847
:1097380093F83C30012B01D1022360E07B680122C1
:1097480083F83C20FB6823F0FF023B68DB68134387
:10975800FB60FB6823F440723B689B681343FB6023
:10976800FB6823F480623B685B681343FB60FB681B
:1097780023F400623B681B681343FB60FB6823F417
:1097880080523B681B691343FB60FB6823F400525B
:109798003B685B691343FB60FB6823F480423B68CA
:1097A8009B6A1343FB60FB6823F470223B689B6948
:1097B8001B041343FB607B681B68144A934215D152
:1097C800FB6823F470023B685B6A1B051343FB606C
:1097D800FB6823F080723B68DB691343FB60FB681E
:1097E80023F000723B681B6A1343FB607B681B68AD
:1097F800FA685A647B68002283F83C2000231846E4
:109808001437BD465DF8047B704700BF002C01404B
:10981800DFF834D0FBF784FA0C480D490D4A0023D1
:1098280002E0D458C4500433C4188C42F9D30A4A0D
:109838000A4C002301E013600432A242FBD300F07B
:1098480011F8F9F71DFCFEE7008000200000002059
:10985800680000206899000868000020880400203B
:10986800FEE7000070B50D4D0D4C641BA4100026DA
:10987800A64209D10B4D0C4C00F046F8641BA4100D
:109888000026A64205D170BD55F8043B984701361D
:10989800EEE755F8043B98470136F2E7609900086F
:1098A800609900086099000864990008024403461A
:1098B800934200D1704703F8011BF9E710EE103A04
:1098C800C3F3C7527F3A162A194615DC002A0CDB67
:1098D8000C481041184205D04FF4800313410B4443
:1098E80023EA000300EE103A7047013203F0004308
:1098F800F8D143F07E53F5E7802AF3D130EE000A21
:10990800704700BFFFFF7F00F8B500BFF8BC08BC78
:109918009E467047F8B500BFF8BC08BC9E46704725
:10992800FFFFFFFFFFFF0000000000000000000035
:1099380001020304060708090203040506070809CB
:109948000A0B0C0D0E0F1010010203040506070880
:08995800090A0B0C0D0E0F10A3
:04996000BD0A000834
:04996400950A000858
:109968000D000000B80B000000000000160D0000FC
:10997800000020417A0D00000000A041AC0D00005D
:109988000000F041CA0D000000002042F20D000066
:1099980000004842100E0000000070422E0E000029
:1099A80000008C42740E00000000A042D80E000097
:1099B8000000B442221000000000C84200127A00E1
:0899C800100000000100000086
:04000005080098193E
:00000001FF
